:100000000C94FC3D0C946E3E0C946E3E0C946E3E33
:100010000C946E3E0C946E3E0C946E3E0C946E3EB0
:100020000C946E3E0C946E3E0C946E3E0C946E3EA0
:100030000C946E3E0C94D13E0C94103F0C946E3E8A
:100040000C946E3E0C946E3E0C946E3E0C946E3E80
:100050000C946E3E0C946E3E0C946E3E0C946E3E70
:100060000C946E3E0C946E3E0C946E3E0C946E3E60
:10007000615961596359665969596C596F595A5593
:10008000012001010038080000000000000000000D
:1000900000000000000000000000000000008100DF
:1000A00045005DFF5E1027FF2AD22B7D210C22FB2D
:1000B000850084008903888D81096F0244424700CE
:1000C0004501B083B300B10124B925578A1D8B03C4
:1000D0008C428F42904294429B42A342A842AD423E
:1000E000B042C042C342C642014304430743000238
:1000F0000800085504085A0000F8000990000A1E7C
:1001000032050000FF000000EE00000000000000CB
:1001100000000000000000000000000000000000DF
:1001200000000000000000000000000000000000CF
:1001300000000000000000000000000000000000BF
:1001400000000000000000000000000000000000AF
:10015000000000000000000000000000000000009F
:100160000049000000495252000052525C2D00002C
:10017000000000000000000000000000000000403F
:10018000000000494A52004952525B1C52531C2540
:10019000241B2425251B0A0A2D1C12120A0A000002
:1001A000000000000000404949494949525B5B5B3F
:1001B000525B1C1C1312241C12090909120909099B
:1001C000090A0A0A0A0A0A13120A0A12130A000082
:1001D0000000000092525252525213121309001C96
:1001E0000A1212401B65090A0009241B120000258F
:1001F0001C1C010025241C1C002425242424000090
:10020000000000005249494000001B1352494900B8
:10021000641C1C5B4A481C651C2552491C1C652437
:1002200064491C1C652564491C1C6D2E5C4900003A
:1002300000000000000000000049000000005352D0
:1002400000000053522500004A52252500005B257E
:100250001300005B53000A1C095B1C657F3740528A
:10026000522E2E1C525C2E251B1324251C1C120002
:100270002525120000121B0000132E37001B3737F4
:100280002E2E37372E2E2E2E2E2E6E6E6E1C131304
:10029000120009131200001213130012251C13136D
:1002A0002E371C131313361C131B1B1B25131C1C6E
:1002B0001B1B1B1C1C1C1C1C1C1C1C1C1C1313129D
:1002C000121313001313131C000913131C0100371E
:1002D000131C13002E2E1C1C001C772E2500137FD0
:1002E000251C010A37241C1C0A2E25250900132E63
:1002F000242525252E252525252525252D2E251B9F
:100300002E2E251C1325251C1C1C1C011C1C130037
:10031000011C0A000165775C016E7F6E521B25256A
:100320006D1C524925251C1353001C1C1C524A00ED
:100330001B135B5B000009525C0000005B5C00006B
:1003400000001B0000000000000000000000135B24
:100350007F776E6E136577766E6E1B657776767631
:100360001B5BBF76B67609136DBFB7B6001B125C78
:1003700076BF0000121B125B00000000090A6E6EBF
:100380006E77241C6E6E77251C1C6E776E1C1C1CF1
:1003900076761C1C2425B765646D6D1B766D6D5BD0
:1003A00009125B5C5B125B641213131B12121C1CA0
:1003B0001C1C1C241C1C242525242425251B000072
:1003C0002513000064BF00096EBFBF6D6EBF6D5B7B
:1003D00012135B12131209000901000000002E1C09
:1003E0000900096E010009767F7F12777F7F641212
:1003F000BF775B121B095B121B0900001B09000081
:1004000000000000000000000000000000007F7FEE
:100410005313130064121B0100001B1200000000A4
:1004200000000000000000000000000000000000CC
:1004300000000000000000000000000000000000BC
:10044000000000002600000026002F0000002F0002
:10045000370000003700FF000000FF00BF00000071
:10046000BF00370000370000002626000000000013
:1004700000000000262626262600000000002F008F
:100480000000003700000000FF00000000BF000077
:100490000000370000000000262626262600000067
:1004A000000000002626262626002F00000000005F
:1004B000370000000000FFFFFFFF0000BF0000004A
:1004C0000000370000000000262626262600000037
:1004D000000000002626262600002F0000002F0026
:1004E000370000003700FFFFFFFF0000BF000000E3
:1004F000BF00370000003700262626260000000037
:1005000000000000000026262600002F00002F001B
:10051000370000003700FF000000FF00BF000000B0
:10052000BF0037000037000026262600000000002C
:10053000000000002600000026002F0000002F0011
:100540000037003700000000FF00000000BF00BFC0
:1005500000003700000037002600000026000000E1
:10056000000000000000000000000000000000008B
:10057000000000000000000000000000000000007B
:10058000009B000000529BA400005B9B6D77000065
:100590000000000000000000000000000000005B00
:1005A000000000E4F6FF099BEDF6FFBFA4ADBFBF5E
:1005B000BFBF767F7FB7B7BF7F766EB7B7BF00008C
:1005C0000000000000005BB6F6F6F6FFFFFFFFBF7D
:1005D000FFFFFFBFBFAEFFFFFFB7AD65FFFFB7B6C1
:1005E000AD65FFFFBFB7AE6EFFFFBFB7B7650000D9
:1005F00000000000F6F6EDEDADA4B66D6D5C526E38
:100600006565655265765C5C52536E246552526E28
:1006100025255B52772D2525526E6E2D2525000050
:1006200000000000A49B9B4900006564A49B92000D
:100630006D2525649349656E652E9B5224256D2595
:10064000655225246D2D655225256E2E64520000BD
:100650000000000000000000004A000000005B9B5A
:100660000000005B5B2D0000525B2E2E00015B2D15
:100670001C01005C5B014A654A5B1C6E7F77495B2D
:100680009B77776D5B65776E65656D2D25255C5273
:100690002E25130949641C09095C7F7F091C7F7F93
:1006A000777F777F77777F7F7776777F7F6E656ECF
:1006B0006EA4B6FF655BA4B7BFFF526DBFBFBFFF9F
:1006C0007FBFBFBFBFFFBFBFB7BFFFFF7FB7BFBF0A
:1006D000FFFF6EB7BFBFFFFF77BFBFBFFFFFFFFFCB
:1006E000BFBFB75BFFFFBFBFA464FFFFBFADA47F69
:1006F000FFFFBFA4BF7FFFBFADBFBFBFFFB6BFBF80
:10070000BF77F7BFBFBF7777FFBFBFBF64526D7FB3
:100710006E2E2D2D7F766E6E6E2E777777762E1C51
:100720007F776E251C25776525251C096E6E1C09B3
:1007300049255B494A6E7F645377BF775B5C256EC2
:100740006E255B4A25651C1B5B002524245B53003A
:100750001C1B5B5C00000A5B64000000646400001A
:1007600000005C00000000000000000000005B5C76
:100770007FBF77765C6D7FB777775C6D7FBF77776C
:100780005C64BFBFBFBF0A5C6EBFBFBF0065646D66
:10079000BFBF00005B6D646D00000000125B7777E7
:1007A000777F6E6E77777F766D7677BF776D6E76B3
:1007B000BF7F6D6E767FBF7676BFBF76BFBFBFB699
:1007C00064ADADB6B6ADBFFF646DADB6AD6477BF19
:1007D000BFBFFFFF77BFBFBFFFFF7FBFBFBFFFF63A
:1007E000BFB7ADF6FFFFA4ADFFFFFFFFFFFFFFFFA9
:1007F000FFFFFFFFFFF6A4005B5200000000BFBF39
:10080000AD5B64BFB6ADADBFFFBFFFFFFFFFBF6411
:10081000FFFFBFB6765BFFBFBF5B0000FF5C000061
:100820000000000000000000000000000000BFBF4A
:10083000645C5C006E5C654900006D5B000000005C
:1008400000000000000000000000000000000000A8
:10085000000000000000000000000000000006048E
:10086000000102030405060708090A0B0C0D0E0F10
:1008700010001112131415160603001718191A1B6D
:100880001C1D1E1F202122232425260000408891A4
:10089000D2E4ADB5B6BEBFFFFFFFFFFFFFFFFFFF16
:1008A000FFFFFFFFFFFFFFFFFFFFFFFFFFFFFFFF58
:1008B000FFFFFFFFFFFFFFFFFFFFFFFFFFFFFFFF48
:1008C000FFFFFFFFFFFFFFFFFFFF00000000FFFF34
:1008D00000000000FFFF00000000FFFF000000001C
:1008E000FFFF00000000FFFF00000000FFFF00000E
:1008F0000000FFFF00000000FFFFFFFFFFFFFFFF02
:10090000FFFFFFFFFFFFFFFFFFFFFFFFFFFFFFFFF7
:10091000FFFFFFFF0000FFFFFF000000FFFF0000E0
:100920000000FFFF00000000FFFF00000000FFFFCD
:1009300000000000FFFF00000000FFFF00000000BB
:100940000000FFFFFFFF0000FFFFFFFF0000FFFFB1
:10095000FFFF0000FFFFFFFF00000000000000009D
:100960000000000000000000000000000000000087
:10097000000000000000FF0000000000FFFF00007A
:100980000000FFFF00000000FFFFFFFFFFFFFFFF71
:10099000FFFFFFFFFFFFFFFFFFFFFFFFFFFFFF0066
:1009A000FFFFFFFF0000FFFFFF000000FFFF000050
:1009B0000000FFFF00000000FFFFFFFFFFFFFFFF41
:1009C000FFFFFFFFFFFFFFFFFFFF00000000000031
:1009D0000000000000000000000000000000000017
:1009E0000000000000000000FFFF00000000FFFF0B
:1009F00000000000FFFF00000000000000000000F9
:100A000000000000000000000000000000000000E6
:100A100000000000000000000000FFFFFFFF0000DA
:100A2000FFFFFFFF0000FFFFFFFF0000FFFFFFFFD2
:100A30000000FFFFFFFF0000FFFFFFFF0000FFFFC0
:100A4000FFFF0000FFFFFFFFFFFF00000000FFFFB0
:100A500000000000FFFF00000000FFFFFFFFFFFF9E
:100A6000FFFFFFFFFFFFFFFFFFFFFFFFFFFFFFFF96
:100A7000FFFFFFFFFFFFFFFF00000000000000007E
:100A800000000000000000000000FFFFFFFFFF006B
:100A9000FFFFFFFFFFFFFFFFFFFFFFFFFFFFFFFF66
:100AA000FFFFFFFFFFFFFFFFFFFFFF000000FFFF53
:100AB000FF000000FFFFFFFF0000FFFFFFFF00003F
:100AC000FFFFFFFFFF00FFFFFFFFFF00FFFFFFFF34
:100AD000FFFFFFFFFFFFFFFFFFFFFFFFFFFFFFFF26
:100AE000FFFFFFFFFFFFFFFFFFFFFFFFFFFFFFFF16
:100AF000FFFFFFFFFF00FFFFFFFFFF00FFFFFFFF04
:100B00000000FFFFFFFF0000FF0000000000FF00EB
:100B100000000000000000000000000000000000D5
:100B200000000000000000000000000000000000C5
:100B30000000000000000000000000000000FF00B6
:100B400000000000FF0000000000FF0000000000A7
:100B5000FFFF00000000FFFF00000000FFFF00009B
:100B60000000FFFF00000000FFFFFFFF0000FFFF8D
:100B7000FF000000FFFFFF000000FFFFFF0000007C
:100B8000FFFF00000000FFFF00000000FFFF00006B
:100B90000000FFFF00000000FFFF00000000FFFF5B
:100BA000FF000000FFFFFF000000FFFFFF0000004C
:100BB000FFFFFF000000FFFF00000000FF0000003B
:100BC0000000FF0000000000FFFF00000000FF0029
:100BD00000000000FF0000000000FF000000000017
:100BE000FF0000000000FFFF00000000FFFFFF000B
:100BF0000000FFFFFF000000FFFFFFFFFFFFFFFF00
:100C0000FFFFFFFFFFFFFFFFFFFFFFFFFFFFFFFFF4
:100C1000FFFFFFFFFFFFFFFFFFFFFF00FFFFFFFFE3
:100C20000000FFFF00000000FFFF00000000FFFFCA
:100C300000000000FFFF00000000FF0000000000B7
:100C400000000000000000000000000000000000A4
:100C50000000000000000000FFFF00000000FFFF98
:100C600000000000FFFF00000000FFFFFF00000089
:100C7000FFFFFFFF0000FFFFFFFFFF00FFFFFFFF81
:100C8000FFFFFFFFFFFFFFFF00000000000000006C
:100C90000000000000000000000000000000000054
:100CA0000000000000000000000000000000000044
:100CB0000000FFFF00000000FFFFFFFFFFFFFFFF3E
:100CC000FFFFFF00FFFFFFFFFF00FFFFFFFFFFFF32
:100CD000FFFFFFFFFFFFFFFFFFFFFFFFFFFFFFFF24
:100CE000FFFFFFFFFFFFFFFF00000000000000000C
:100CF00000000000000000000000000000000000F4
:100D0000FFFFFF000000FFFFFFFFFFFFFFFFFFFFF0
:100D1000FFFFFFFFFFFFFFFF0000000000000000DB
:100D200000000000000000000000000000000000C3
:100D3000000000000000FFFF00000000FFFFFFFFB9
:100D40000000FFFFFF000000FFFFFFFFFFFFFFFFAE
:100D5000FFFFFFFFFFFFFFFFFFFFFFFFFFFFFFFFA3
:100D6000FFFFFFFFFFFFFFFF00000000000000008B
:100D70000000FF0000000000FFFFFFFF0000FFFF7A
:100D8000FFFFFF00FFFFFFFFFF00FFFFFFFF00006F
:100D9000FF00000000000000000000000000000054
:100DA0000000000000000000FFFFFF000000FFFF48
:100DB000FFFF0000FFFFFFFFFF00FFFFFFFFFF003F
:100DC000FFFFFFFFFF00FFFFFFFFFF00FFFFFFFF31
:100DD000FF00FFFFFFFFFF00FFFFFFFFFFFFFFFF21
:100DE000FFFFFFFFFFFFFFFFFF00FFFFFFFFFF0011
:100DF000FFFFFFFFFF00FFFFFFFFFF00FFFFFFFF01
:100E0000FF00FFFFFFFFFF00FF00000000000000E9
:100E100000000000000000000000000000000000D2
:100E200000000000000000000000000000000000C2
:100E300000000000000000000000000000000000B2
:100E40000000000000000000000000FFFFFF0000A5
:100E5000FFFFFFFF0000FFFFFFFF0000FFFFFFFF9E
:100E60000000FFFFFFFF0000000000000000000086
:100E70000000000000000000000000000000000072
:100E8000000000000000000000FFFFFF0000FFFF67
:100E9000FFFF00FFFFFFFFFF000000000000000059
:100EA0000000000000000000000000000000000042
:100EB000000000000000FF0000000000FF00000034
:100EC0000000FF0000000000000000000000000023
:100ED000000000000000000000000000000000FF13
:100EE00000000000FFFF00000000FFFF0000000006
:100EF000FFFF00000000FFFF0000000000000000F6
:100F000000000000000000000000FFFF00000000E3
:100F1000FFFF00000000FFFF00000000FFFF0000D7
:100F20000000FFFF00000000FFFFFFFFFF00FFFFCA
:100F3000FFFFFF00FFFFFFFFFF00FFFFFFFFFF00BE
:100F4000FFFFFFFFFF00FFFFFFFFFF00FFFFFFFFAF
:100F5000FF00FFFFFFFF0000FFFFFFFFFF00FFFF9D
:100F6000FFFFFF00FFFFFFFFFF00FFFFFFFFFF008E
:100F7000FFFFFFFFFF00FFFFFFFFFF00FFFFFFFF7F
:100F8000FF00FFFFFFFFFFFF000000000000000068
:100F90000000000000000000000000000000000051
:100FA0000000000000000000000000FF0000000042
:100FB00000FF0000000000FF000000000000000033
:100FC00000FFFFFF00FFFFFFFFFFFFFFFFFFFFFF2F
:100FD000FFFFFFFFFF00FFFFFFFF0000FFFFFF001D
:100FE0000000FFFFFF000000000000000000FFFF06
:100FF00000000000FFFFFF000000FFFFFF000000F7
:1010000000000000000000000000000000000000E0
:101010000000000000000000FFFFFFFF0000FFFFD6
:10102000FFFFFFFFFFFFFFFFFFFFFFFFFFFFFFFFD0
:10103000FFFFFFFF0000FFFFFFFF0000FFFFFFFFBC
:101040000000FFFFFFFF0000000000000000FFFFA6
:1010500000000000FFFFFFFF0000FFFFFFFF000098
:10106000FFFFFFFFFF0000FFFFFFFF0000FFFFFF8C
:10107000FF0000FFFFFFFF00000000000000000075
:10108000000000FF000000FFFFFF0000FFFFFFFF68
:101090000000FFFFFFFF00FFFFFFFF0000FFFFFF5B
:1010A000FF0000FFFFFFFFFF000000000000FFFF48
:1010B000FFFF0000FFFFFFFFFF00FFFFFFFFFFFF3D
:1010C0000000FFFFFFFF000000FFFFFF000000FF28
:1010D000FFFFFFFFFFFFFFFF000000000000000018
:1010E0000000000000000000FFFF000000FFFFFF05
:1010F000000000FFFFFFFF0000FFFFFFFF0000FFF9
:10110000FFFFFF000000FFFF000000000000FFFFE6
:10111000FFFFFFFFFFFFFFFFFFFFFFFFFFFFFFFFDF
:10112000FF0000000000FF0000000000FFFFFFFFC5
:10113000FFFFFFFFFFFFFFFF0000000000000000B7
:101140000000000000000000FFFF000000FFFFFFA4
:10115000000000FFFFFF000000FFFFFF000000FF96
:10116000FFFF00000000FFFF000000000000000083
:10117000000000000000000000FF0000000000FF71
:1011800000000000FFFF00000000FFFF000000FF64
:10119000FFFF000000FFFFFF00FFFFFFFFFFFFFF5B
:1011A000FFFFFFFFFFFF00FFFFFFFFFF00FFFFFF4D
:1011B000FF0000FFFFFFFF0000FFFFFFFF0000FF39
:1011C000FFFFFFFFFFFFFFFFFF0000000000FF0029
:1011D00000000000FF0000000000FF000000000011
:1011E000FF0000000000FF0000000000FF00000002
:1011F0000000FFFFFF000000000000000000FFFFF4
:10120000FFFF0000FFFFFFFF0000FFFFFFFF0000E8
:10121000FFFFFFFF0000FFFFFFFF0000FFFFFFFFDA
:101220000000FFFFFFFF000000000000000000FFC3
:10123000FFFFFF0000FFFFFFFF0000FFFFFFFF00B9
:1012400000FFFFFFFF0000FFFFFFFF0000FFFFFFA9
:10125000FF0000FFFFFFFF0000000000000000FF94
:10126000FFFFFFFF00FFFFFFFFFF00FFFFFFFFFF8C
:101270000000000000FF0000000000FF0000000070
:10128000FFFF000000FFFFFF000000000000FFFF65
:10129000FFFFFF00FFFFFFFFFF00FFFFFFFFFF005B
:1012A000FFFFFFFF0000FFFFFFFF0000FFFFFF0049
:1012B0000000FFFF0000000000000000FFFF000032
:1012C0000000FFFF00000000FFFF00000000FFFF24
:1012D00000000000FFFFFF000000FFFFFF00000014
:1012E000FFFFFF000000FFFFFFFF00000000FFFF07
:1012F000FFFFFFFFFFFFFFFFFFFFFFFFFFFFFFFFFE
:10130000FFFF000000FFFFFF00000000FFFF0000E4
:101310000000FFFF00000000000000000000FF00D0
:1013200000000000FFFF00000000FFFFFF000000C2
:10133000FFFFFF000000FFFFFFFF0000FFFFFFFFB8
:101340000000FFFFFFFF00000000000000000000A1
:101350000000FFFF0000FFFFFFFF00FFFFFFFFFF98
:1013600000FFFFFFFFFFFFFFFFFFFF00FFFFFFFF8B
:101370000000FFFFFFFF0000000000000000FFFF73
:10138000FF000000FFFFFFFFFF00FFFFFFFFFFFF69
:1013900000FFFFFFFFFF0000FFFFFFFF000000FF57
:1013A000FFFF000000FFFFFF000000000000000042
:1013B000FFFFFFFF000000FFFFFF00000000FFFF36
:1013C00000000000FFFFFF00000000FFFF00000022
:1013D0000000FF0000000000000000000000FF000F
:1013E0000000FFFFFF000000FFFFFFFF00FFFFFF07
:1013F000FFFFFFFFFFFFFFFFFFFFFFFFFFFFFFFFFD
:10140000FF00FFFFFFFFFF00000000000000FFFFE4
:10141000FF000000FFFF00000000FF0000000000D0
:1014200000000000000000000000000000000000BC
:101430000000000000000000FFFFFFFF0000FFFFB2
:10144000FFFF0000FFFFFFFF0000FFFFFFFF0000A6
:10145000FFFFFFFF0000FFFFFFFF0000FFFFFFFF98
:101460000000FFFFFFFF00000000000000FF000081
:10147000000000FF0000000000000000000000006D
:10148000000000000000000000000000000000005C
:101490000000000000000000FFFFFF000000FFFF51
:1014A000FFFF0000FFFFFFFFFF00FFFFFFFFFFFF49
:1014B00000FFFFFFFFFF000000FFFFFF0000000034
:1014C000000000000000000000000000000000001C
:1014D00000000000000000000000FFFFFF0000000F
:1014E000FFFFFF000000FFFF000000000000000001
:1014F0000000000000000000FFFFFFFF0000FFFFF2
:10150000FFFF0000FFFFFFFF0000FFFFFFFF0000E5
:10151000FFFFFFFF0000FFFFFFFF000000000000D3
:10152000000000000000000000FFFFFFFF0000FFC0
:10153000FFFFFF0000FFFFFFFF0000FFFFFFFF00B6
:1015400000FFFFFFFF0000FFFFFFFF0000000000A3
:10155000000000000000000000FFFFFFFFFF00FF91
:10156000FFFFFF000000FFFFFFFF0000FFFFFFFF86
:10157000000000FFFFFF0000000000FF000000006F
:101580000000000000000000FFFFFFFFFFFF000061
:1015900000000000000000000000FFFFFFFFFFFF51
:1015A000FFFFFFFFFFFFFFFFFFFFFF000000000046
:1015B0000000000000000000FF00000000FF00002D
:1015C00000000000000000FF0000000000FFFFFF1F
:1015D000000000FFFFFF00000000FFFF0000000010
:1015E0000000000000000000FFFFFFFFFFFF000001
:1015F000FFFFFFFF000000FFFFFFFFFFFFFFFFFFF8
:10160000FFFFFFFFFFFFFFFFFFFF000000000000E4
:101610000000000000000000FF00000000FFFF00CD
:1016200000000000FF0000FF0000FF0000FFFFFFC0
:10163000000000FFFFFF00000000FFFF00000000AF
:101640000000000000000000FF0000FFFFFFFF009F
:1016500000FFFFFFFF0000000000FF00000000008F
:10166000000000000000000000000000000000007A
:101670000000000000000000FFFFFFFFFFFFFFFF72
:10168000FFFFFFFF000000FFFFFF000000FFFFFF64
:10169000000000FFFFFF000000FFFFFF0000000050
:1016A0000000000000000000FFFFFF000000FFFF3F
:1016B000FF000000FF0000000000FF00000000002D
:1016C000FF0000000000FF0000000000000000001C
:1016D0000000000000000000FFFFFFFF0000FFFF10
:1016E000FFFF0000FFFFFFFFFF0000FFFFFFFFFF06
:1016F00000FFFFFFFFFF000000FFFFFF00000000F2
:10170000000000000000000000FFFFFFFF0000FFDE
:10171000FFFFFF0000FFFFFFFF00FFFFFFFFFF00D5
:10172000FFFFFFFFFF00FFFFFFFF000000000000C2
:101730000000000000000000000000FFFFFF0000AC
:10174000FFFFFFFF0000FFFFFFFF00FFFFFFFFFFA6
:1017500000FFFFFFFFFF00FFFFFFFFFF0000000093
:101760000000000000000000FFFF00000000FF007C
:1017700000000000FF0000000000FFFFFFFFFF006F
:10178000FFFFFFFFFF00FFFFFFFFFF000000000063
:101790000000000000000000FF000000FFFF00004C
:1017A0000000FFFF00000000FFFF00000000FFFF3F
:1017B00000000000FFFF0000000000FF000000002C
:1017C0000000000000000000FFFF00000000FFFF1D
:1017D000000000FFFFFF0000FFFFFFFFFFFFFFFF14
:1017E000FFFFFFFFFFFFFFFFFFFFFFFF0000000005
:1017F0000000000000000000FFFFFFFF0000FFFFEF
:10180000FFFF0000FFFFFF000000FFFFFF000000E0
:10181000FFFF0000000000000000000000000000CA
:101820000000000000000000FFFFFFFF0000FFFFBE
:10183000FFFFFF0000FFFFFFFFFF00FFFFFFFFFFB5
:101840000000FFFFFFFF00000000FFFF000000009E
:101850000000000000000000000000FFFFFF00008B
:10186000FFFFFFFF00FFFFFFFFFFFFFFFFFFFFFF87
:10187000FFFFFFFFFF00FFFFFF0000000000000070
:101880000000000000000000FF0000000000FF005A
:10189000000000FF00000000FFFF00000000FFFF4D
:1018A000000000FFFFFF0000FFFFFFFF000000003F
:1018B0000000000000000000FFFFFFFFFF00FFFF2F
:1018C000FFFFFFFFFFFFFFFFFFFFFFFF00FFFFFF27
:1018D000FFFF00FFFFFFFF000000FFFF0000000010
:1018E00000000000000000000000000000000000F8
:1018F00000000000FF0000000000FF0000000000EA
:10190000FFFF00000000FFFFFF00000000000000DC
:101910000000000000000000FFFFFFFF0000FFFFCD
:10192000FFFF0000FFFFFF000000FFFFFF000000BF
:10193000FFFFFF000000FFFFFF000000FFFFFF00B0
:101940000000FFFFFF00000000000000000000009A
:1019500000000000FF0000000000FF000000000089
:10196000FF0000000000FF0000000000FF0000007A
:101970000000FF0000000000FFFFFF000000FFFF6D
:10198000FF000000FFFFFF000000FFFFFF0000005E
:10199000FFFF00000000FFFF00000000FFFF00004D
:1019A0000000FFFF00000000FF0000000000FF003B
:1019B00000000000FF0000000000FF000000000029
:1019C000FFFF00000000FFFF00000000FFFF00001D
:1019D0000000FFFF00000000FFFF00000000FF000C
:1019E00000000000FF0000000000FF0000000000F9
:1019F000FF000000000000000000000000000000E8
:101A00000000000000000000FFFF00000000FFFFDA
:101A1000FF000000FFFFFF000000FFFFFF000000CD
:101A2000FFFFFF000000FFFFFFFF0000FFFFFFFFC1
:101A30000000FFFFFFFF0000FFFFFFFFFFFFFFFFB2
:101A4000FFFFFF00FFFFFFFFFF00FFFFFFFFFF00A3
:101A5000FFFFFFFF0000FFFFFFFF0000FFFFFFFF92
:101A60000000FFFFFF000000FFFFFFFF0000FFFF7F
:101A7000FFFFFF00FFFFFFFFFF00FFFFFFFFFF0073
:101A8000FFFFFFFFFFFFFFFFFFFFFFFFFFFFFFFF66
:101A9000FFFFFFFFFFFFFFFF00000000000000004E
:101AA0000000000000000000000000000000000036
:101AB0000000000000000000000000000000000026
:101AC0000000FF0000000000FFFFFFFFFFFFFFFF1F
:101AD000FFFFFFFFFFFFFFFFFFFFFFFFFFFFFFFF16
:101AE000FFFFFFFFFFFFFFFFFFFFFFFFFFFFFFFF06
:101AF000FFFFFFFFFFFFFF00FFFFFF000000FFFFF2
:101B000000000000FFFF00000000FF0000000000D8
:101B1000FF0000000000FF000000000000000000C7
:101B20000000000000000000FF0000000000FFFFB8
:101B300000000000FFFF00000000FFFFFF000000AA
:101B4000FFFFFF000000FFFFFF000000FFFFFFFF9F
:101B50000000FFFFFFFFFF00FFFFFFFFFF00FFFF91
:101B6000FFFFFF00FFFFFFFF0000FFFFFFFF000080
:101B7000FFFFFF000000FFFFFF000000FFFF00006D
:101B80000000FFFF00000000FFFFFFFFFF00FFFF5E
:101B9000FFFFFF00FFFFFFFFFFFFFFFFFFFFFFFF54
:101BA000FFFFFFFFFFFFFFFFFFFFFFFFFFFFFFFF45
:101BB000FFFFFFFFFFFFFFFF00000000000000002D
:101BC0000000000000000000000000000000000015
:101BD000FF0000000000FF0000000000FFFF000009
:101BE0000000FFFF00000000FFFFFFFFFFFFFFFFFF
:101BF000FFFFFFFFFFFFFFFFFFFFFFFFFFFFFF00F4
:101C0000FFFFFFFF0000FFFFFFFF0000FFFFFF00DF
:101C10000000FFFFFF000000FFFFFF000000FFFFCC
:101C2000FFFF0000FFFFFFFF0000FFFFFFFFFF00BF
:101C3000FFFFFFFFFFFFFFFFFFFFFFFFFFFFFFFFB4
:101C4000FFFFFFFFFFFFFFFF00000000000000009C
:101C50000000000000000000000000000000000084
:101C6000000000000000000000000000FF00000075
:101C70000000FF0000000000FFFF00000000FFFF69
:101C800000000000FFFF00000000FFFF0000000058
:101C9000FFFF00000000FFFF00000000FFFFFF004B
:101CA0000000FFFFFFFF0000FFFF00000000FFFF3C
:101CB00000000000FFFF00000000FFFF0000000028
:101CC000FFFF00000000FFFF00000000FF00000019
:101CD0000000000000000000000000000000000004
:101CE00000000000000000000000000000000000F4
:101CF00000000000000000000000000000000000E4
:101D00000000000000000000000000FF00000000D4
:101D1000FFFFFF000000FFFFFF00000000FF0000CA
:101D2000000000FF0000000000000000000000FFB5
:101D3000000000000000000000FFFF00FFFF00FFA8
:101D4000FF00FFFF00FF0000FF0000000000000098
:101D50000000000000000000000000000000000083
:101D60000000000000000000000000000000000073
:101D7000FF00FF0000FFFFFFFFFF0000FF00FF006C
:101D80000000FF00FF0000FFFFFFFFFF0000FF005B
:101D9000FF000000000000000000FF000000000045
:101DA000FFFFFF0000FF000000000000FFFF000039
:101DB00000000000FF0000FFFFFF0000000000FF28
:101DC000000000000000000000FFFF0000FF00FF17
:101DD000FF0000FF00000000FF00000000FF000007
:101DE0000000FF00000000FF0000FFFF00FF0000F8
:101DF000FFFF0000000000000000FF00000000FFE7
:101E000000FF000000FF00FF00000000FF000000D6
:101E100000FF00FF00FF00FF0000FF000000FFFFC9
:101E200000FF0000000000000000FFFF00000000B5
:101E3000FFFF00000000FF000000000000000000A5
:101E40000000000000000000000000000000000092
:101E50000000000000000000000000FF0000000083
:101E6000FF0000000000FF0000000000FF00000075
:101E70000000FF0000000000FF000000000000FF65
:101E800000000000000000000000FF000000000053
:101E900000FF0000000000FF0000000000FF000045
:101EA000000000FF0000000000FF00000000FF0035
:101EB0000000000000000000000000000000000022
:101EC000FF00FF000000FFFFFF0000FFFFFFFFFF1C
:101ED0000000FFFFFF000000FF00FF000000000007
:101EE00000000000000000000000000000000000F2
:101EF00000FF0000000000FF000000FFFFFFFFFFE9
:101F0000000000FF0000000000FF000000000000D3
:101F100000000000000000000000000000000000C1
:101F200000000000000000000000000000000000B1
:101F30000000000000000000FFFF00000000FFFFA5
:101F400000000000FF000000000000000000000092
:101F50000000000000000000000000FFFFFFFFFF86
:101F60000000000000000000000000000000000071
:101F70000000000000000000000000000000000061
:101F80000000000000000000000000000000000051
:101F90000000000000000000FFFF00000000FFFF45
:101FA0000000000000000000000000000000000031
:101FB000000000FF00000000FF00000000FF000024
:101FC0000000FF00000000FF000000000000000013
:101FD00000000000000000000000FFFFFF0000FF05
:101FE000000000FF00FF0000FFFF00FF00FF00FFF8
:101FF00000FFFF0000FF00FF000000FF0000FFFFE8
:10200000FF00000000000000000000FF00000000D2
:10201000FFFF0000000000FF0000000000FF0000C4
:10202000000000FF0000000000FF00000000FFFFB4
:10203000FF000000000000000000FFFFFF0000FFA5
:10204000000000FF0000000000FF000000FFFF0094
:102050000000FF00000000FF0000000000FFFFFF85
:10206000FFFF0000000000000000FFFFFF0000FF76
:10207000000000FF0000000000FF0000FFFFFF0065
:102080000000000000FF00FF000000FF0000FFFF55
:10209000FF0000000000000000000000FF00000042
:1020A00000FFFF000000FF00FF0000FF0000FF0036
:1020B00000FFFFFFFFFF00000000FF000000000026
:1020C000FF0000000000000000FFFFFFFFFF00FF17
:1020D0000000000000FF0000000000FFFFFFFF0005
:1020E0000000000000FF00FF000000FF0000FFFFF5
:1020F000FF00000000000000000000FFFF000000E3
:10210000FF00000000FF0000000000FFFFFFFF00D5
:1021100000FF000000FF00FF000000FF0000FFFFC5
:10212000FF0000000000000000FFFFFFFFFF0000B5
:10213000000000FF00000000FF00000000FF0000A2
:102140000000FF0000000000FF0000000000FF0092
:1021500000000000000000000000FFFFFF0000FF83
:10216000000000FF00FF000000FF0000FFFFFF0075
:1021700000FF000000FF00FF000000FF0000FFFF65
:10218000FF000000000000000000FFFFFF0000FF54
:10219000000000FF00FF000000FF0000FFFFFFFF46
:1021A0000000000000FF00000000FF000000FFFF33
:1021B000000000000000000000000000000000001F
:1021C000000000000000FFFF00000000FFFF000013
:1021D0000000000000000000FFFF00000000FFFF03
:1021E00000000000000000000000000000000000EF
:1021F000000000000000FFFF00000000FFFF0000E3
:102200000000000000000000FFFF00000000FFFFD2
:1022100000000000FF00000000000000FF000000C0
:1022200000FF00000000FF00000000FF00000000B1
:102230000000FF000000000000FF000000000000A0
:10224000FF0000000000000000000000000000008F
:102250000000000000FFFFFFFFFF00000000000083
:1022600000000000000000FFFFFFFFFF0000000073
:1022700000000000000000000000FF00000000005F
:1022800000FF000000000000FF000000000000FF51
:1022900000000000FF00000000FF00000000FF0041
:1022A00000000000000000000000FFFFFF0000FF32
:1022B000000000FF0000000000FF000000FFFF0022
:1022C000000000FF0000000000000000000000FF10
:1022D00000000000000000000000FFFFFF0000FF02
:1022E000000000FF00FF00FFFFFF00FF00FF00FFF6
:1022F00000FF00FFFFFF00FF000000000000FFFFE5
:10230000FF000000000000000000FFFFFF0000FFD2
:10231000000000FF00FF000000FF00FF000000FFC2
:1023200000FFFFFFFFFF00FF000000FF00FF0000B5
:1023300000FF00000000000000FFFFFFFF0000FFA3
:10234000000000FF00FF000000FF00FFFFFFFF0094
:1023500000FF000000FF00FF000000FF00FFFFFF84
:10236000FF000000000000000000FFFFFF0000FF72
:10237000000000FF00FF0000000000FF0000000060
:1023800000FF0000000000FF000000FF0000FFFF52
:10239000FF0000000000000000FFFFFFFF0000FF43
:1023A000000000FF00FF000000FF00FF000000FF32
:1023B00000FF000000FF00FF000000FF00FFFFFF24
:1023C000FF0000000000000000FFFFFFFFFF00FF14
:1023D0000000000000FF0000000000FFFFFFFF0002
:1023E00000FF0000000000FF0000000000FFFFFFF2
:1023F000FFFF00000000000000FFFFFFFFFF00FFE5
:102400000000000000FF0000000000FFFFFFFF00D1
:1024100000FF0000000000FF0000000000FF0000BF
:1024200000000000000000000000FFFFFF0000FFB0
:10243000000000FF00FF0000000000FF00FFFFFFA2
:1024400000FF000000FF00FF000000FF0000FFFF92
:10245000FFFF00000000000000FF000000FF00FF81
:10246000000000FF00FF000000FF00FFFFFFFFFF74
:1024700000FF000000FF00FF000000FF00FF000061
:1024800000FF0000000000000000FFFFFF00000050
:1024900000FF0000000000FF0000000000FF00003F
:1024A000000000FF0000000000FF00000000FFFF30
:1024B000FF000000000000000000000000FF00001E
:1024C000000000FF0000000000FF0000000000FF0F
:1024D00000FF000000FF00FF000000FF0000FFFF02
:1024E000FF0000000000000000FF000000FF00FFF0
:1024F0000000FF0000FF00FF000000FFFF000000E1
:1025000000FF00FF000000FF0000FF0000FF0000D0
:1025100000FF00000000000000FF0000000000FFBE
:102520000000000000FF0000000000FF00000000AD
:1025300000FF0000000000FF0000000000FFFFFFA0
:10254000FFFF00000000000000FF000000FF00FF90
:10255000FF00FFFF00FF00FF00FF00FF000000FF83
:1025600000FF000000FF00FF000000FF00FF000070
:1025700000FF00000000000000FF000000FF00FF5F
:10258000FF0000FF00FF00FF00FF00FF0000FFFF53
:1025900000FF000000FF00FF000000FF00FF000040
:1025A00000FF0000000000000000FFFFFF0000FF30
:1025B000000000FF00FF000000FF00FF000000FF20
:1025C00000FF000000FF00FF000000FF0000FFFF11
:1025D000FF0000000000000000FFFFFFFF0000FF01
:1025E000000000FF00FF000000FF00FFFFFFFF00F2
:1025F00000FF0000000000FF0000000000FF0000DE
:1026000000000000000000000000FFFFFF0000FFCE
:10261000000000FF00FF000000FF00FF000000FFBF
:1026200000FF00FF00FF00FF0000FF000000FFFFB1
:1026300000FF00000000000000FFFFFFFF0000FFA0
:10264000000000FF00FF000000FF00FFFFFFFF0091
:1026500000FF0000FF0000FF000000FF00FF00007F
:1026600000FF0000000000000000FFFFFF0000FF6F
:10267000000000FF00FF000000000000FFFFFF005F
:102680000000000000FF00FF000000FF0000FFFF4F
:10269000FF0000000000000000FFFFFFFFFF000040
:1026A00000FF0000000000FF0000000000FF00002D
:1026B000000000FF0000000000FF0000000000FF1D
:1026C000000000000000000000FF000000FF00FF0D
:1026D000000000FF00FF000000FF00FF000000FFFF
:1026E00000FF000000FF00FF000000FF0000FFFFF0
:1026F000FF0000000000000000FF000000FF00FFDE
:10270000000000FF00FF000000FF00FF000000FFCE
:1027100000FF000000FF0000FF00FF00000000FFBE
:10272000000000000000000000FF000000FF00FFAC
:10273000000000FF00FF00FF00FF00FF00FF00FFA0
:1027400000FF00FF00FF00FF00FF00FF0000FF0090
:10275000FF0000000000000000FF000000FF00FF7D
:10276000000000FF0000FF00FF00000000FF00006D
:102770000000FF00FF0000FF000000FF00FF00005E
:1027800000FF00000000000000FF000000FF00FF4D
:10279000000000FF00FF000000FF0000FF00FF003E
:1027A000000000FF0000000000FF0000000000FF2C
:1027B000000000000000000000FFFFFFFF0000001D
:1027C0000000FF00000000FF00000000FF0000000C
:1027D00000FF0000000000FF0000000000FFFFFFFE
:1027E000FF000000000000000000FFFFFF000000ED
:1027F000FF0000000000FF0000000000FF000000DC
:102800000000FF0000000000FF0000000000FFFFCC
:10281000FF0000000000000000000000000000FFBA
:10282000000000000000FF000000000000FF0000AA
:1028300000000000FF000000000000FF000000009A
:1028400000000000000000000000FFFFFF0000008B
:102850000000FF0000000000FF0000000000FF007B
:1028600000000000FF0000000000FF000000FFFF6C
:10287000FF00000000000000000000FF000000005A
:10288000FF00FF0000FF000000FF0000000000004C
:102890000000000000000000000000000000000038
:1028A0000000000000000000000000000000000028
:1028B0000000000000000000000000000000000018
:1028C0000000000000000000000000000000000008
:1028D0000000FFFFFFFFFFFF0000FFFF0000000000
:1028E000FFFF0000000000FF0000000000000000EB
:1028F00000000000000000000000000000000000D8
:1029000000000000000000000000000000000000C7
:10291000000000000000FFFFFF000000000000FFBB
:102920000000FFFFFFFF00FF000000FF0000FFFFAF
:10293000FFFF00000000000000FF0000000000FF9B
:102940000000000000FFFFFFFF0000FF000000FF8D
:1029500000FF000000FF00FF000000FF00FFFFFF7E
:10296000FF00000000000000000000000000000068
:10297000000000000000FFFFFF0000FF000000FF5C
:1029800000FF0000000000FF000000FF0000FFFF4C
:10299000FF000000000000000000000000FF000039
:1029A000000000FF0000FFFFFFFF00FF000000FF2E
:1029B00000FF000000FF00FF000000FF0000FFFF1D
:1029C000FFFF000000000000000000000000000009
:1029D000000000000000FFFFFF0000FF000000FFFC
:1029E00000FFFFFFFF0000FF000000000000FFFFEE
:1029F000FF00000000000000000000FFFF000000DA
:102A0000FF0000000000FF00000000FFFFFFFF00CC
:102A10000000FF0000000000FF0000000000FF00B9
:102A200000000000000000000000000000000000A6
:102A3000000000000000FFFFFFFF00FF000000FF9C
:102A400000FF000000FF0000FFFFFFFF000000008C
:102A500000FF0000FFFFFF0000FF0000000000FF7C
:102A60000000000000FFFFFF000000FF0000FF006B
:102A700000FF0000FF0000FF0000FF0000FF00005B
:102A8000FF00000000000000000000FF0000000048
:102A900000000000000000FF0000000000FF000038
:102AA000000000FF0000000000FF0000000000FF29
:102AB000FF0000000000000000000000FF00000018
:102AC00000000000000000FFFF0000000000FF0009
:102AD00000000000FF0000000000FF0000FF0000F9
:102AE000FF000000FFFF000000FF0000000000FFEB
:102AF0000000000000FF0000FF0000FF00FF0000DA
:102B000000FFFF00000000FF00FF000000FF0000CA
:102B1000FF00000000000000000000FF00000000B7
:102B200000FF0000000000FF0000000000FF0000A8
:102B3000000000FF0000000000FF0000000000FF98
:102B4000FF00000000000000000000000000000086
:102B50000000000000FFFF00FF0000FF00FF00FF7B
:102B600000FF00FF00FF00FF000000FF00FF00006B
:102B700000FF000000000000000000000000000056
:102B80000000000000FFFFFF000000FF0000FF004A
:102B900000FF0000FF0000FF0000FF0000FF00003A
:102BA000FF00000000000000000000000000000026
:102BB000000000000000FFFFFF0000FF000000FF1A
:102BC00000FF000000FF00FF000000FF0000FFFF0B
:102BD000FF000000000000000000000000000000F6
:102BE0000000000000FFFFFFFF0000FF000000FFEB
:102BF00000FF000000FF00FF000000FF00FFFFFFDC
:102C0000FF0000FF000000000000000000000000C6
:102C1000000000000000FFFFFFFF00FF000000FFBA
:102C200000FF000000FF00FF000000FF0000FFFFAA
:102C3000FFFF0000000000FF000000000000000097
:102C40000000000000FF00FFFF000000FF0000FF89
:102C50000000FF0000000000FF00000000FFFFFF79
:102C60000000000000000000000000000000000064
:102C7000000000000000FFFFFF0000FF0000000058
:102C80000000FFFFFF000000000000FF0000FFFF4A
:102C9000FF00000000000000000000000000000035
:102CA000FF00000000FFFFFFFF000000FF0000002A
:102CB0000000FF0000000000FF00FF00000000FF18
:102CC0000000000000000000000000000000000004
:102CD0000000000000FF0000FF0000FF0000FF00F8
:102CE00000FF0000FF0000FF00FFFF000000FF00EA
:102CF000FF000000000000000000000000000000D5
:102D00000000000000FF000000FF00FF000000FFC7
:102D100000FF000000FF0000FF00FF00000000FFB8
:102D200000000000000000000000000000000000A3
:102D30000000000000FF000000FF00FF000000FF97
:102D400000FF00FF00FF00FFFFFFFFFF0000FF008C
:102D5000FF00000000000000000000000000000074
:102D60000000000000FF0000FF0000FF0000FF0067
:102D70000000FFFF000000FF0000FF0000FF000058
:102D8000FF00000000000000000000000000000044
:102D90000000000000FF0000FF0000FF0000FF0037
:102DA00000FF0000FF000000FFFFFF00000000FF29
:102DB000000000FFFF000000000000000000000015
:102DC0000000000000FFFFFFFF0000000000FF0008
:102DD0000000FFFF000000FF0000000000FFFFFFF9
:102DE000FF00000000000000000000FFFF000000E6
:102DF000FF0000000000FF00000000FFFF000000D7
:102E00000000FF0000000000FF000000000000FFC5
:102E1000FF00000000000000000000FF00000000B4
:102E200000FF0000000000FF0000000000000000A4
:102E3000000000FF0000000000FF0000000000FF95
:102E400000000000000000000000FFFF0000000084
:102E50000000FF0000000000FF0000000000FFFF76
:102E600000000000FF0000000000FF000000FFFF66
:102E700000000000000000000000FF00FF0000FF55
:102E800000FF000000000000000000000000000043
:102E90000000000000000000000000000000000032
:102EA0000000000000000000000000FF0000000023
:102EB000FFFFFF0000FFFF00FFFF00FF000000FF1B
:102EC00000FF000000FF00FFFFFFFFFF0000000009
:102ED0000000000000000000C7C7C7C7C7C7C7C7BA
:102EE000C7C7C7C7C7C7C7C7C7C7C7C7C7C7C7C772
:102EF000C7C7C7C7C7C7C7C7C7C7C7C7C7C7C7C762
:102F0000C7C7C7C7C7C7C7C7281C00000000000045
:102F1000000000016C6C6C6C6C6C6C6C6C6C6C6CA0
:102F20006C6C6C6C6C6C6C6C6C6C6C6C6C6C6C6CE1
:102F30006C6C00000000000000000203046C6C6C6C
:102F40006C6C6C6C6C6C6C6C6C6C6C6C6C6C6C6CC1
:102F50006C6C6C6C6C6C6C6C6C6C00000000000039
:102F600005060708090A046C6C6C6C6C6C6C6C6C64
:102F70006C6C6C6C6C6C6C6C6C6C6C6C6C6C6C6C91
:102F80006C6C0000000000000B6C6C08000C0D6CF9
:102F90006C6C6C6C6C6C6C6C6C6C6C6C6C6C6C6C71
:102FA0006C6C6C6C6C6C6C6C6C6C000000000000E9
:102FB000000E6C08000F6C6C6C6C6C6C6C6C6C6C48
:102FC0006C6C6C6C6C6C6C6C6C6C6C6C6C6C6C6C41
:102FD0006C6C00000000000000106C0800116C6CAC
:102FE0006C6C6C6C6C6C6C6C6C6C6C6C6C6C6C6C21
:102FF0006C6C6C6C6C6C6C6C6C6C00000000000099
:1030000012136C080014156C6C6C6C6C6C6C6C6C32
:103010006C6C6C6C6C6C6C6C6C6C6C6C6C6C6C6CF0
:103020006C6C00000000001617186C0800191A6C70
:103030006C6C6C6C6C6C6C6C6C6C6C6C6C6C6C6CD0
:103040006C6C6C6C6C6C6C6C6C6C00000000000048
:10305000001B6C081C1D6C6C1E6C6C6C6C6C6C6CBE
:103060006C1F206C6C6C6C6C6C21226C6C6C6C6CCE
:103070006C6C00000000000000236C08242526274B
:1030800028292A2B2C2D2E2D2F3031323334352A5E
:103090002B363738393A3B3C3D6C000000000000CD
:1030A000003E6C08003F4041424344454647484784
:1030B000494A4B4C4D4E4F4445505152535455562E
:1030C000576C00000000000000586C0800596C6C40
:1030D0006C6C6C6C6C6C6C6C6C6C6C6C6C6C6C6C30
:1030E0006C6C6C6C6C6C6C6C6C6C000000000000A8
:1030F000005A6C08005B6C6C6C6C6C6C6C6C6C6C6F
:103100006C6C6C6C6C6C6C6C6C6C6C6C6C6C6C6CFF
:103110006C6C000000000000005C6C08005D6C6CD2
:103120006C6C6C6C6C6C6C6C6C6C6C6C6C6C6C6CDF
:103130006C6C6C6C6C6C6C6C6C6C00000000000057
:103140005E6C6C08005F606C6C6C6C6C6C6C6C6CB6
:103150006C6C6C6C6C6C6C6C6C6C6C6C6C6C6C6CAF
:103160006C6C000000000061626C6C080000636C15
:103170006C6C6C6C6C6C6C6C6C6C6C6C6C6C6C6C8F
:103180006C6C6C6C6C6C6C6C6C6C000000000064A3
:103190006C6C6C08000065666C6C6C6C6C6C6C6CB8
:1031A0006C6C6C6C6C6C6C6C6C6C6C6C6C6C6C6C5F
:1031B0006C6C00000000671D6C6C6C0800000068FF
:1031C000696C6C6C6C6C6C6C6C6C6C6C6C6C6C6C42
:1031D0006C6C6C6C6C6C6C6C6C6C000000006A6CE1
:1031E0006C6C6C08000000006B6C6C6C6C6C6C6C34
:1031F0006C6C6C6C6C6C6C6C6C6C6C6C6C6C6C6C0F
:103200006C6C000000000000000000016C6C6C6C35
:103210006C6C6C6C6C6C6C6C6C6C6C6C6C6C6C6CEE
:103220006C6C6C6C6C6C6C6C6C6C00000000000066
:10323000000000016C6C6C6C6C6C6C6C6C6C6C6C7D
:103240006C6C6C6C6C6C6C6C6C6C6C6C6C6C6C6CBE
:103250006C6C000000000000000000016C6C6C6CE5
:103260006C6C6C6C6C6C6C6C6C6C6C6C6C6C6C6C9E
:103270006C6C6C6C6C6C6C6C6C6C00000000000016
:10328000000000016C6C6C6C6C6C6C6C6C6C6C6C2D
:103290006C6C6C6C6C6C6C6C6C6C6C6C6C6C6C6C6E
:1032A0006C6C000000000000000000016C6C6C6C95
:1032B0006C6C6C6C6C6C6C6C6C6C6C6C6C6C6C6C4E
:1032C0006C6C6C6C6C6C6C6C6C6C000000000000C6
:1032D000000000016C6C6C6C6C6C6C6C6C6C6C6CDD
:1032E0006C6C6C6C6C6C6C6C6C6C6C6C6C6C6C6C1E
:1032F0006C6C000000000000000000016C6C6C6C45
:103300006C6C6C6C6C6C6C6C6C6C6C6C6C6C6C6CFD
:103310006C6C6C6C6C6C6C6C6C6C00000000000075
:10332000000000016C6C6C6C6C6C6C6C6C6C6C6C8C
:103330006C6C6C6C6C6C6C6C6C6C6C6C6C6C6C6CCD
:103340006C6C000000000000000000016C6C6C6CF4
:103350006C6C6C6C6C6C6C6C6C6C6C6C6C6C6C6CAD
:103360006C6C6C6C6C6C6C6C6C6C00000000000025
:10337000000000000000000000000000000000004D
:10338000000000000000000000000000000000003D
:10339000000000000000000000000000000000002D
:1033A000000000000000000000000000000000001D
:1033B000000000000000000000000000000000000D
:1033C0000000000000000000003F000000000000BE
:1033D0000000003F0000003F0000373700000037CA
:1033E00037370000373737373F0037070707000008
:1033F000370737373F00373737373F0000000000C7
:103400003F00003F0000373700000000373737002B
:10341000003F373737370000373737370000073777
:10342000373737003707073700000000000000007B
:103430000000000000000000000000003F0000004D
:1034400000000000000000003F000000000000003D
:10345000000000000000000000000000000000006C
:103460000000000000000000000000000000FFFF5E
:10347000FFFF0000FFFFFFFF0000000000FF000053
:10348000000000FF0000000000FF0000000000003E
:10349000000000000000000000000000FFFFFFFF30
:1034A000FFFFFFFFFFFFFFFFFFFF00000000FFFF28
:1034B00000000000FFFF000000000000000000000E
:1034C0000000000000000000000000000000FFFFFE
:1034D000000000FFFFFF000000FFFFFF000000FFF3
:1034E000FFFFFFFF00FFFFFFFFFF000000000000E5
:1034F00000000000000000000000000000000000CC
:103500000000000000000000000000000000FFFFBD
:1035100000000000FFFFFF0000FF000000000000AF
:10352000000000000000000000000000FFFFFF009E
:103530000000FFFF00000000000000000000FFFF8F
:10354000000000FFFFFF0000FFFF00000000000080
:10355000000000000000000000000000000000006B
:103560000000000000000000000000000000FF005C
:10357000FFFFFFFFFFFFFFFFFFFF00000000000055
:10358000000000000000000000000000000000003B
:10359000FFFF000000FFFFFF000000FFFFFF000033
:1035A00000FFFFFF000000FFFF0000000000000020
:1035B000000000000000000000000000000000000B
:1035C00000000000000000000000000000000000FB
:1035D000FFFFFF0000FFFF000000000000000000F0
:1035E00000000000000000000000000000FFFFFFDE
:1035F000000000FFFF00000000000000000000FFCE
:10360000FF000000FFFFFF0000FF000000000000BF
:1036100000000000000000000000000000000000AA
:103620000000000000000000000000000000FFFF9C
:1036300000FFFFFFFFFFFFFFFFFF00000000000093
:10364000000000000000000000000000000000007A
:103650000000000000000000000000000000FF006B
:10366000000000FFFF000000FFFF0000000000005E
:10367000000000000000000000000000000000004A
:103680000000000000000000000000000000FFFF3C
:10369000FFFFFFFFFFFFFFFFFFFF0000370037378F
:1036A00000373700373700370037370000373737F4
:1036B0000037F7F73700370000F7F7F70000F7F7A4
:1036C000F7F70000000000000000373F3737000028
:1036D00000003700000037370000003F0000000006
:1036E00000000000003F000000000000000000009B
:1036F00000000000000000000000003F000000008B
:1037000000000000000000000000000000000000B9
:1037100000000000000000000000000000000000A9
:10372000000000000000000000000000000000FF9A
:103730000000000000FF00000000FFFF000000008C
:10374000FFFF00000000FFFF00000000FFFF00007F
:1037500000000000000000000000FFFF000000006B
:10376000FF0000000000FF0000000000FF0000005C
:103770000000FF0000000000FF000000000000004B
:103780000000000000000000000000FFFFFF00003C
:1037900000FFFF000000FFFFFF000000FFFFFF0031
:1037A0000000FFFF000000FFFFFF000000FF00001F
:1037B00000000000000000000000FFFFFF0000FF0D
:1037C000FFFFFF0000FFFFFF000000FFFFFF000002
:1037D00000FFFFFF0000FFFFFFFF0000FFFF0000F2
:1037E00000000000000000000000FFFF0000FFFFDD
:1037F000FFFF0000FFFFFF000000FFFFFF000000D1
:10380000FFFFFF0000FFFFFFFF0000FFFFFF0000C2
:1038100000000000000000000000FF000000FFFFAB
:10382000FF0000FFFFFF000000FFFFFF000000FFA0
:10383000FFFF000000FFFF00000000FFFF0000008E
:1038400000000000000000000000000000FFFFFF7B
:10385000000000FFFFFF0000FFFFFFFF0000FFFF71
:10386000FF000000FFFF00000000FFFF000000005D
:1038700000000000000000000000FFFF000000004A
:10388000FF0000000000FFFF00000000FFFFFF003E
:10389000000000FFFF0000FF00FFFFFF00FF00002F
:1038A00000000000000000000000FFFF000000FF1B
:1038B000FFFF0000FFFFFF000000FFFFFF00000010
:1038C000FFFFFF000000FFFFFF000000FFFF000000
:1038D00000000000000000000000FF0000FFFFFFEC
:1038E000FF0000FFFFFFFF0000FFFF00FF0000FFE1
:1038F000FFFF000000FFFFFF00000000FFFF0000CF
:1039000000000000000000FFFFFF000000FFFFFFBD
:10391000000000FFFF00000000FFFF000000FFFFAD
:10392000FF00FFFFFFFFFF00FF00FFFF000000FFA1
:10393000FFFF0000FFFFFF0000000000000000008C
:103940000000000000000000000000000000FFFF79
:1039500000000000FFFF000000FFFFFF000000006C
:103960000000000000000000000000000000000057
:1039700000000000000000000000000000FFFFFF4A
:10398000000000FFFFFF000000FFFFFF000000003D
:103990000000000000000000000000000000000027
:1039A00000000000000000000000000000FFFF0019
:1039B000000000FFFF000000FFFFFF00000000000C
:1039C00000000000000000000000C7C7C7C7C7C74D
:1039D000C7C7C7C7C7C7C7C7C7C7C7C7C7C7C7C777
:1039E000C7C7C7C7C7C7C7C7C7C7C7C7C7C7C7C767
:1039F000C7C7C7C7C7C7C7C7C7C7280200000000D7
:103A00000000000000000102030405060708090A7F
:103A10000B0C0D0E0F100000000000000000000055
:103A20000000000000000000000000000000001185
:103A300012131415161718191A1B171C1D1E1F20F8
:103A40002100000000000000000000000000000055
:103A50000000000000000000000000000000000066
:103A60000000000000000000000000000000000056
:103A7000000000000000000000000000B7B77777EA
:103A8000B7B7B77777B7B7B77777B7B7B777B7B706
:103A9000B7777777B7B77777B7B7B77777B7B7B776
:103AA0007777B7B7B725B7B7B777771CB7B7777753
:103AB000B7B7B77777B7B7B77777B7B7B777B7B7D6
:103AC000B7777777B7251C1C25B72577BFBF372574
:103AD00077BFFFBFBFB7BFFFFFBFBF77B7B777776E
:103AE000B7B7B77777B7B7B77777B7B7B777B7B7A6
:103AF000B7777777B7B77777B7B7B77777B7B7B716
:103B00002577B7B7B7771CB7B7777777B7B7777732
:103B1000B7B7B77777B7B7B77777B7B7B777B7B775
:103B2000B7251C6EB7B7771CBF77B777771CBF7701
:103B30007777B71CBF77B7B7B725BFBFB7B777776A
:103B4000B7B7B77777B7B7B77777B7B7B777771C20
:103B50001C1C1C7765BFBFBF776565BFFFBF77655E
:103B600065BFFFBF7765B7BFFFBFBFB7B7B7777791
:103B7000B7B7B77777B7B7B77777B7B7B7776E1CF9
:103B800025777777BF771C77B7B7BF771CB7B7B7FD
:103B9000BF771CB7B777BF7725777777B7B77777D2
:103BA000B7B7B77777B7B7B77777B7B7B777B7B7E5
:103BB000B7777777B7B77777B7B7B77777B7251C82
:103BC0007777B72577B7B7B7B71CFF7FB7B77777E2
:103BD000B7B7B77777251C257777B71C7777B7B74F
:103BE00025FF7FB7251CBF256EBFB7FFBFB777BFC7
:103BF000FF7FBFBFBFBF7FBFBFBFBFBFB7B77777B5
:103C0000B7B7B77777B7B7B72577B7B7B7771C6EBA
:103C1000B777777777256E77B7B7BF6E1C6EB7B774
:103C2000BF77251CB777BFB7251C7777B7B77777EE
:103C3000B7B7B77777B7B7B77777B7B7B777B7B754
:103C4000B7777777B7B77777B76EB77777B76E1CF1
:103C50007777B7B72577B7B7B7771CBFB7B7777799
:103C6000B7B7B777251CB7B77725BFBF6577B71C40
:103C700065651CB71C6EBFBF771C77656EBFBF77CD
:103C8000BF77656EBF77BFBF77BFBF77B7B77777AF
:103C9000B7B7B77777B7B7B77777B7B7B777B7B7F4
:103CA000B77777776EB77777B7B7256E77B7B7B748
:103CB000251CB7B7B777251CB7777777B7B777776E
:103CC000B7B7B77777B7B7B77777B7B7B777B7B7C4
:103CD000B7777777B7B777252E25B777771C7F77B4
:103CE0007777B71C77BFB7B7B76E1C7FB7B7251C00
:103CF000B7B7B725BFBF65B7771C65651C7725BF0C
:103D0000FFB777257765B7666577FFB7776EFF777B
:103D1000FFFFBFBFBFB7BF7FBFBFBFB7B7B7777723
:103D2000B7B7B77777B7B7B77777B7B7B777B7B763
:103D3000B7777777252E2577B7B7FF251CB7B7B7A5
:103D400077251CB7B7776E1C6E777777B7B777771D
:103D5000B725B77777B7B7B77777B7B7B72EB7B70E
:103D6000B777771CB7B77777B72EB77777B7B777C7
:103D70007777B7B7B777B7B7B7777725B7BFBFBF8D
:103D8000372E2E77B7372E1D25656565652577BFDC
:103D9000FFBF772E252E6E2E25251CB7B76E2E1C45
:103DA00025FFBF776E1C2EFFBF776E2525B777776F
:103DB000B7B7777777B7B7B72EB7B7B7B7771CB7B7
:103DC000B77777772EB77777B7B7777777B7B7B70C
:103DD0007777B7B7B7772EB7B7777777B7B77777FC
:103DE00025BFB77777B76E657777B7B7B71CB7B723
:103DF000B777771CB7B77777B71CB77777B76E25E4
:103E00007777B7B71C6EB7B7B7771C77BFBFBFBFA1
:103E1000BFBF656E776E65656EB7B7B76E6E77BFFD
:103E2000FFBF776E77BFFFBF776E77BFFFBF776E3D
:103E3000B7BFFFBF776E7FBFFFBFB76E77257777BE
:103E4000B7B7666E77B7B7B71C77B7B7B7771CB792
:103E5000B77777771CB77777B7B7256E77B7B7B7E8
:103E6000251CB7B7B7772E1CB7777777B7B7B71CCE
:103E70007777B777776E1C1C7777B7B7B777B7B711
:103E8000B777776EB7B777776E25B777776E257781
:103E90007777B7257777B7B7B71C7777656E77B73A
:103EA000BFBF6E656E7FBFFF251DB7FFFFBF1D77CC
:103EB000FFFFBFB7777FFFFFBFB7B7FFFFFFBF773A
:103EC000B7FFFFBFBF6E7FFFFFBFB76EBFB7251C39
:103ED000B7B7B7B71C6EB7B7B7771CB7B777772543
:103EE0006E7777776E1C7777B7B76E1C77B7B7B7F3
:103EF0006E1CB7B7B7776E256E777777B7B77777DA
:103F00001CBFB77777B76E257777B7B7B71CB7B74A
:103F1000B7776E1CB7B77777B71CB77777B7251D1C
:103F20007777B7B71C6EB7B7B76E1C77BFBFBFBF89
:103F3000B76EBFBFBF776E25656E776E656577BF5D
:103F4000FFBF776666666E6666256EB7B7B76E6E3C
:103F5000B7BFFFBF776E7FBFFFBFB76E251C7777F8
:103F6000B7B7256E77B7B7B71C77B7B7B7771C6EFB
:103F7000B77777771CB77777B7B71D2577B7B7B718
:103F80006E1CB7B7B7776E1C6E777777B7B7777752
:103F90002577B77777B7651C7777B7B76E1CB7B754
:103FA000B777B71CB7B777776E1DB77777B7256543
:103FB0007777B7B71C6EB7B7B76E1C77BFBFBF7741
:103FC0006E25656E776E656577BFFFBF776666663F
:103FD0006E6666666EB7B7B76E6EB7BFFFBF776EB9
:103FE000B7BFFFBF776E7FBFFFBFB76E1C25777768
:103FF000B7B71C6577B7B7B71C6EB7B7B7771CB73D
:10400000B77777771D6E7777B7B7652577B7B7B787
:104010006E1CB7B7B7776E1C6E777777B7B77777C1
:104020002E1CB77777B725777777B72E1C7FB7B772
:10403000B71CBF2EB7B7771C77BFB77777B7251CEC
:104040007777B7B7B777B7B7B777777777FFBF77B0
:104050006E2E7FFFBFB76E6EFFFFBFB76E6E25255A
:104060002E252525FFFFBFBF77771C1C1C1C1C1CA1
:104070002E2E2E2E2E2EB7B7B77777771C2E77776A
:10408000B7B71C25B7B7B7B72E1C2EB7B7772525FE
:104090001C77777725251C77B7B71C2577B7B7B777
:1040A0007777B7B7B777B7B7B7777777B7B7771CFB
:1040B0006E77B777251C657F77771CBF776EB7B7AC
:1040C0001C77BFBFB7B7256E6E6EB77777251C1C00
:1040D0007777B7B7B725B7B7B77777777FFFFFBFE2
:1040E000B76E7FFFFFBFB76E25252E252525FFFF65
:1040F000BFBFBF776E6E6E6E6E6E1C1C1C1C1C1CD0
:10410000252525252525B7B7B77777776E25257718
:10411000B7B76E251C25B7B76E6E251CB7777777B6
:10412000251C77776E256525B7B71C1C25B7B7B753
:104130002577B7B7B777B7B7B7777777B7B7777761
:10414000B7B7B77777B7B7B77777B7B7B777B7B73F
:10415000B777776EB7B7776E251CB77777257F77F8
:104160007777B71C77BFB7B7B76E1C7FB76EFFBF47
:104170006EB72525FFBF25256EFFFFBFBF6E6EBF43
:10418000BF77776E6565BF7725657725BF7725771C
:10419000FF256E6E6EB7BF7FBFBFBFB7B7B777776C
:1041A000B7B7B77777B7B7B77777B7B7B7776EB728
:1041B000B77777771C1D6E77B7B7FF2525B7B7B7E9
:1041C00077251CB7B7776E1C6E77777726266666DD
:1041D000662666666626262666662626666666263F
:1041E000266626262626665D251C2666661C7F77A3
:1041F0006666261C77BF6626261D657F266EFFBF76
:104200006E262525FFBF25256EFFFFBFBF6E6EBF43
:10421000BF77776E6565BF7725657725BF7725778B
:10422000FF256E6E6EB7BF7FBFBFBFB7262666661F
:10423000662666666626262666662626666626261E
:10424000266666661C1D5D666666FF251C6626265C
:1042500077251C2666666E651D6666662626661CC4
:104260006E7766665D1C657F66661CBF776E662628
:104270001C77BFBF26261D6E6E6E6666661D1C1CF3
:1042800066662626661D6626266666667FFFFFBF73
:10429000B76E7FFFFFBFB76E25252E252525FFFFB3
:1042A000BFBFBF776E6E6E6E6E6E1C1C1C1C1C1C1E
:1042B0001D1D1D1D1D1D6626266666666E251D2696
:1042C00066266E251C1D26266E6E251C6666777773
:1042D000251C66666E25651D66261C1C1D26262669
:1042E0001D66262666666626266666662626666637
:1042F000662666666626262666662626666666261E
:10430000266666662626666666266666662626260D
:1043100066662626661D66262666661C2626666650
:1043200066266666662626266666262666666626ED
:1043300026666666261D1C1C1D261D77BFBF371D01
:1043400077BFFFBFBFB7BFFFFFBFBF772626666639
:1043500066266666662626266666262666666626BD
:1043600026666666262666666626666666262626AD
:104370001D66262666661C262666666626266666F0
:10438000662666666626262666662626666666268D
:10439000261D1C652626661CBF776666661CBF77D1
:1043A0006666261CBF776626261DBFBF2626666664
:1043B0006626666666262626666626266666661C67
:1043C0001C1C1C6665BFBFBF776565BFFFBF7765F7
:1043D00065BFFFBF7765B7BFFFBFBFB7262666665D
:1043E0006626666666262626666626266666651C38
:1043F0001D666666BF771C666626BF771C26262666
:10440000BF771C266666BF771D66666626266666CB
:1044100066266666662626266666262666666626FC
:1044200026666666262666666626666666261D1CFF
:104430006666261D77B76626261CFF7F26266666DB
:1044400066266666661D1C1D66661D1C7777661DE2
:104450006EFF7FB71D1CBF256EBFB7FFBFB777BF0D
:10446000FF7FBFBFBFBF7FBFBFBFBFBF2626666680
:1044700066266666662626261D66262666661C1D38
:104480002666666677251D666626BF6E1C2626266E
:10449000BF77251D6666BFB7251C6666262666663D
:1044A000662666666626262666662626666666266C
:1044B0002666666626266666662666666626261D65
:1044C000666626261D77662626661CBF2626666635
:1044D000662666661D1C2626661DBFBF6566661CB1
:1044E00065656E661D6EBFBF771D77656EBFBF7752
:1044F000BF77656EBF77BFBF77BFBF77262666667B
:10450000662666666626262666662626666666260B
:10451000266666662626666666261D666626262644
:10452000251D26266666251C266666662626666680
:1045300066266666662626266666262666666626DB
:10454000266626262626661D2E252666661C7F776D
:104550006666261C77BF6626261D657F26661D1C9F
:104560002626661DBFBF6526661C65656E661DBF77
:10457000FFB7771D7765B7666577FFB7776EFF770B
:10458000FFFFBFBFBFB7BF7FBFBFBFB726266666EF
:1045900066266666662626266666262666662626BB
:1045A00026666666252E1D666666FF251C6626261F
:1045B00077251C2666666E651D6666662626666617
:1045C000661D66666626262666662626661D66269D
:1045D0002666661C26266666661D6666662626268E
:1045E00066662626666666262666661C1D2666663E
:1045F00066262666662626261D66262666661C26EE
:10460000266666661D266666662666666626262613
:104610006666262666661D26266666662626665D0C
:104620002EBF666666261D6566662626661C66269D
:104630002666661C26266666661C666666261D2538
:10464000666626261C6E6626261D1C77772E5D66FE
:104650006626651D662626261C66262666661C2698
:10466000266666661C2666666626251D662626263E
:10467000251C262666662E1C5D6666662626661C3A
:1046800077776666661D1C1C666626266666662645
:10469000266666652626666665256666662625772D
:1046A0006666261D77776626261C7777656E77B750
:1046B000BFBF66656E7FBFFF651DB7FFFFBF1D777C
:1046C000FFFFBFB7777FFFFFBFB7B7FFFFFFBF7722
:1046D000B7FFFFBFBF6E7FFFFFBFB76EBFB7251C21
:1046E0006626B7B71C652626B7771C26666677252B
:1046F000656666666E1C666666266E1C66262626DF
:104700006E1C262666666E251D666666262666660D
:104710001CBF666666261D7766662626661C6626AC
:1047200026661D1C26266666661C666666261D6550
:10473000666626261C6E6626261D1C77251C666668
:104740006626251D662626261C66262666661C1DF0
:10475000266666661C2666666626651D662626260D
:104760006E1C262666666E1C5D6666662626666676
:104770001D7766666626661C666626261D1C6626EE
:104780002666661C262666661D65666666261C6E9F
:10479000666626261C6E6626261D1C77251D666607
:1047A00066261C66662626261C1D262666661C2690
:1047B00026666666651D666666266E1C6626262665
:1047C0006E1C262666666E1C5D666666B7B77777D2
:1047D000B7B7B77777B7B7B77777B7B7B777B7B7A9
:1047E000B7777777B7B77777B7B7B77777B7B76E62
:1047F0007777B7B7B713B7B7B7777701B7B7777723
:10480000B7B7B77777B7B7B77777B7B7B777B7B778
:10481000B77777776E0A01010A6E01010101010085
:1048200001015C010100015CFF130100B7B777775C
:10483000B7B7B77777B7B7B77777B7B7B777B7B748
:10484000B7777777B7B77777B7B76E7777B7B7B701
:104850001377B7B7B77700B7B7777777B7B7777703
:10486000B7B7B77777B7B7B77777B7B7B777B7B718
:10487000B7130A01B7B777005C09B7777700020969
:104880007777B70A0209B7B7B76E0102B7B777777C
:10489000B7B7B77777B7B7B77777B7B7B7776E0ADE
:1048A0000101016E14005C01091413000A010913CF
:1048B00009000A010909010001010101B7B7777771
:1048C000B7B7B77777B7B7B77777B7B7B7770A021A
:1048D00013777777020A0077B7B7020100B7B7B747
:1048E00002000AB7B77701006E777777B7B77777A7
:1048F000B7B7B77777B7B7B77777B7B7B777B7B788
:10490000B7777777B7B77777B7B7B77777B76E1CDB
:104910007777B76E0A0AB7B7B71C0B00B7B77777C8
:10492000B7B7B777771C0A6E77776E0A090BB76E41
:104930001C0A00026E0B0A000000130A0200130298
:10494000020000020200000000000000B7B7777705
:10495000B7B7B77777B7B7B76E77B7B7B7770A6E26
:10496000B777777700026E77B7B700010A6EB7B7EF
:104970000000016EB7770000020A7777B7B7777744
:10498000B7B7B77777B7B7B77777B7B7B777B7B7F7
:10499000B7777777B7B77777B76EB77777B76E1C94
:1049A0007777B7B71300B7B7B7770A00B7B7777796
:1049B000B7B7B72E000B2EB7770A5C000A776E1DCB
:1049C00000001C6E0A0B020100135C000B020100C8
:1049D0000A5C000B0100000A5C000000B7B77777A3
:1049E000B7B7B77777B7B7B77777B7B7B777B7B797
:1049F000B77777776EB77777B7B71C6E77B7B7B7F4
:104A00000213B7B7B777020AB7777777B7B7777771
:104A1000B7B7B77777B7B7B77777B7B7B777B7B766
:104A2000B777772EB7B777001C01B777770A0213ED
:104A30007777B71C000AB7B7B76E0A02B72E000B1C
:104A40002EB7B70A5C000AB7771300001C770A007C
:104A50000900000A0A010A09010A5C005C13005CF3
:104A6000000000000000090000000000B7B77777E1
:104A7000B7B7B77777B7B7B77777B7B7B7772EB78F
:104A8000B7777777011C0077B7B70B0A0AB7B7B7C4
:104A900000001CB7B777000A6E777777B7B77777DC
:104AA000B713B77777B7B76E7777B7B7B71CB7B71E
:104AB000B7777701B7B77777B713B77777B7B76EA9
:104AC0007777B7B7B76EB7B7B777771C0101130120
:104AD00001001301010100130A000000000A010196
:104AE00001010101000A5C0A00000100010100004F
:104AF00001000A01000001001301000013B77777DD
:104B0000B7B76E7777B7B7B71CB7B7B7B77701B78F
:104B1000B777777713B77777B7B76E7777B7B7B7D2
:104B20006E77B7B7B7771CB7B7777777B7B77777B9
:104B30001C01B77777B76E007777B7B7B700B7B70D
:104B4000B7777700B7B777776E00B77777B71C007E
:104B50007777B7B71C01B7B7B76E00010101010144
:104B6000010100000000000001010101010101003C
:104B70000A000101010013000101010013000001FE
:104B8000000A5C01000200135C010001001C777741
:104B9000B7B7006E77B7B7B70077B7B7B77700B7D3
:104BA000B7777777006E7777B7B7001C77B7B7B767
:104BB000001CB7B7B77701006E777777B7B7B70A3A
:104BC0000000B777776E0A0A7777B7B7B777B7B7C6
:104BD000B777776EB7B777776E00B777776E0A00DB
:104BE0007777B71C0000B7B7B70A00000A0A0000C1
:104BF00000006E1C0A000000770A00000A0A0A0082
:104C00000A135C00000A135C0000000A5C13000138
:104C10000A135C0A00010A13FF0A00010000020ADD
:104C2000B7B70000016EB7B700011CB7B777010A2C
:104C30006E777777010A7777B7B7010A77B7B7B793
:104C400001096EB7B77701001C777777B7B7777729
:104C50000A01B77777B71C007777B7B7B70AB7B746
:104C6000B7771C0AB7B777776500B77777B76E0065
:104C70007777B7B71C01B7B7B76E0A01000001001C
:104C80000001010101010102020A130A02020002ED
:104C90000202010002135C0A02020100130000017B
:104CA000000A5C01000200135C010001020A777730
:104CB000B7B7021C77B7B7B70A77B7B7B7770A1C89
:104CC000B777777700657777B7B7006E77B7B7B7FD
:104CD000001CB7B7B777010A6E777777B7B77777E2
:104CE0001C00B77777B7B70A7777B7B71C0AB7B79B
:104CF000B7776500B7B777776E00B77777B71C00DF
:104D00007777B7B70A01B7B7B76E0A01010101019A
:104D10000102020A130A0202000202020100021347
:104D20005C0A0202010013000101010013000001EE
:104D3000000A5C01000200135C010001021C77778D
:104D4000B7B70AB777B7B7B70A1CB7B7B777006571
:104D5000B7777777006E7777B7B7001C77B7B7B7B5
:104D6000000AB7B7B777010A6E777777B7B7777763
:104D70006E01B77777B71C017777B76E1C00B7B7AE
:104D8000B71C0100B7B777130101B777776E13012E
:104D90007777B7B7B76EB7B7B777777700005C01AB
:104DA0000000000AFF0101000A13130A01000000BD
:104DB00000000000010A130A0101010101010101C3
:104DC0001C1C1C1C1C1CB7B7B7777777006E777755
:104DD000B7B7001CB7B7B7B700006EB7B777000119
:104DE0001C77777701011377B7B701136EB7B7B7A1
:104DF0006E77B7B7B777B7B7B7777777B7B76E0AC2
:104E00000100B7771C01000A77770009010AB7B7DC
:104E100000000913B7B70A010101B7776E1301014A
:104E20007777B7B76E1CB7B7B77777770A13FF0AEC
:104E30000000135CFF0A01000A0A0A0A0A015CFF6B
:104E40005C131309010101010100010101010101CC
:104E50001C1C1C1C1C1CB7B7B777777702000A6EA6
:104E6000B7B70109011CB7B701010000B77700000F
:104E7000000077770001010AB7B70101136EB7B7D9
:104E80001C6EB7B7B777B7B7B7777777B7B7777716
:104E9000B7B7B77777B7B7B77777B7B7B777B7B7E2
:104EA000B7777777B7B7776E1302B777770A0213BA
:104EB0007777B71C0002B7B7B76E0A00B7B70A001A
:104EC000B7B7B7770A00B7B70A0A0A000A0A00009C
:104ED00000000000020A00000B0B020A00000B0099
:104EE0000B030A0A0300130100000000B7B777772D
:104EF000B7B7B77777B7B7B77777B7B7B777B7B782
:104F0000B777777702136E77B7B700000AB7B7B7EE
:104F100000001CB7B777000A6E777777262666669B
:104F200066266666662626266666262666666626E1
:104F3000266666662626661D13026666660A0213E4
:104F40006666261D0002662626660A0026660A0098
:104F5000662666660A0026260A0A0A000A0A000071
:104F600000000000020A00000B0B020A00000B0008
:104F70000B030A0A030013010000000026266666E0
:104F80006626666666262626666626266666662681
:104F90002666666602131D66662600000A26262619
:104FA00000001D266666000A2666666626261D0A1D
:104FB000010066660A01000A66660009010A6626A3
:104FC0000000091326260A01010166661D1301016E
:104FD000666626261D1D6626266666660A13FF0A75
:104FE0000000135CFF0A01000A0A0A0A0A015CFFBA
:104FF0005C1313090101010101000101010101011B
:105000001D1D1D1D1D1D66262666666602000A1DE5
:1050100066260109010A26260101000066660000D5
:10502000000066660001010A66260101131D26269E
:105030001D1D262666666626266666662626666622
:1050400066266666662626266666262666666626C0
:105050002666666626266666666666666626261D79
:1050600066662626660A6626266666012626666621
:105070006626666666262626666626266666662690
:10508000266666661D0A01010A1D01010101010073
:1050900001015C010100015CFF1301002626666628
:1050A0006626666666262626666626266666662660
:1050B000266666662626666666261D666626262699
:1050C0000A662626666600262666666626266666C2
:1050D0006626666666262626666626266666662630
:1050E000260B0A01262666005C0966666600020930
:1050F0006666260A02096626261D010226266666BF
:1051000066266666662626266666262666661D0A64
:105110000101011D14005C01091413000A010913A7
:1051200009000A010909010001010101262666663C
:1051300066266666662626266666262666660A024F
:105140000B666666020A00666626020100262626AF
:1051500002000A26666601001D66666626266666E9
:10516000662666666626262666662626666666269F
:1051700026666666262666666626666666261D0AB4
:105180006666261D0A0A6626260A0B00262666661D
:105190006626666666140A1D66661D0A090B661D8C
:1051A000140A00021D0B0A000000130A0200130279
:1051B00002000002020000000000000026266666D1
:1051C00066266666662626261D66262666660A1DED
:1051D0002666666600021D66662600010A1D2626F2
:1051E0000000011D66660000020A666626266666E5
:1051F000662666666626262666662626666666260F
:105200002666666626266666661D666666261D1323
:10521000666626261300662626660A002626666629
:105220006626661D000B1D26660A5C000A661D13B5
:1052300000000B1D0A0B020100135C000B020100B1
:105240000A5C000B0100000A5C000000262666666E
:1052500066266666662626266666262666666626AE
:10526000266666661D26666666260A1D662626264C
:10527000021326266666020A266666662626666685
:10528000662666666626262666662626666666267E
:105290002666661D262666001C016666660A0213DF
:1052A0006666261D000A662626660A02261D000B73
:1052B0001D26660A5C000A26661300000B660A00BB
:1052C0000900000A0A010A09010A5C005C13005C7B
:1052D00000000000000009000000000026266666AD
:1052E00066266666662626266666262666661D2667
:1052F00026666666011C006666260B0A0A262626B6
:1053000000001D266666000A266666662626666614
:10531000660A66666626261D666626266613662665
:105320002666660126266666661366666626261D5E
:1053300066662626661D66262666660A0A2666664E
:1053400066261D666626262613662626666601667E
:10535000266666661366666666261D6666262626C9
:105360001D66262666660A26266666662626666602
:105370000A01666666261D006666262666006626A3
:1053800026666600262666661D00666666260A0094
:10539000666626260A016626261D0001000A666644
:1053A0006626001D662626260066262666660026D8
:1053B00026666666001D66666626000A662626263E
:1053C000000A2626666601001D6666662626660AAF
:1053D00000006666661D0A0A6666262666666626FA
:1053E00026666613262666661D006666661D0A002A
:1053F0006666261300006626260A00000A0A0000D8
:1054000000001D0B0A000000130A00000A0A0A002F
:105410000A135C00000A135C0000000A5C13000120
:105420000A135C0A00010A13FF0A00010000020AC5
:1054300066260000011D262600010A266666010A6E
:105440001D666666010A66666626010A66262626C7
:1054500001091D26666601001366666626266666D5
:105460000A01666666261D0066662626260A6626E8
:105470002626130A262666661C00666666261D001A
:10548000666626260A016626261D0001020A666651
:105490006626021D662626260A26262666660A1324
:1054A00026666666001C66666626001D662626263B
:1054B000000A2626666601001D6666662626666662
:1054C0001D0066666626260A66662626130A662676
:1054D00026661C00262666666600666666261D0031
:1054E000666626260A016626261D0001021D6666DE
:1054F00066260A26662626260A1326266666001CC7
:1055000026666666002666666626001D66262626D0
:10551000000A2626666601001D666666FFFFFFFF1D
:10552000FFFF373737373737B7B7B7B7B7B737377B
:1055300037373737373737373737373737373737FB
:105540006F6F6F6F6F6F141414141414FFFFFFFF4D
:10555000FFFF372E1C142E37AF1C77AF14B72E0B5E
:10556000372E0B372E0B0B0B0B372E14372E143711
:105570006F6F6F6F6F6F141414141414FFFFFFFF1D
:10558000FFFF2E14141C2E37AF1477AF1DB72E0B50
:105590000B0B26372E0B372E1D372E14141C2E37CF
:1055A0006F6F6F6F6F6F141414141414FFFFFFFFED
:1055B000FFFF372E14142E37AF1D77AF1DB72E0BFC
:1055C000373737372E0B372E1D37372E141C2E3713
:1055D0006F6F6F6F6F6F141414141414FFFFFFFFBD
:1055E000FFFF2E14141C2E37AF1477AF1DB72E0BF0
:1055F000372E0B372E0B372E1D372E14141C2E373B
:105600006F6F6F6F6F6F141414141414FFFFFFFF8C
:10561000FFFF2E1414141437AF1477B7B7B72E0B3F
:105620000B0B37372E0B373737372E14141414372C
:105630006F6F6F6F6F6F141414141414FFFFFFFF5C
:10564000FFFF2E1414141437AF1477B7B7B72E0B0F
:105650000B0B37372E0B373737372E143737373793
:105660006F6F6F6F6F6F141414141414FFFFFFFF2C
:10567000FFFF372E25141437AF1477B7B7B72E0BAB
:10568000370B0B372E14372E1D37372E25141437B2
:105690006F6F6F6F6F6F141414141414FFFFFFFFFC
:1056A000FFFF2E14372E1437AF1477AF14B72E0B1D
:1056B0000B0B0B372E0B372E0B372E14372E1437C0
:1056C0006F6F6F6F6F6F14141414141426266666B0
:1056D0001D2E666666661C776666261D1C7F66261E
:1056E000261CBF2E2626661C77BF666666261D1CF6
:1056F00066662626666666262666666677FFBF7736
:105700006E2E7FFFBFB76E6EFFFFBFB76E6E252593
:105710002E252525FFFFBFBF77771C1C1C1C1C1CDA
:105720001D1D1D1D1D1D6626266666661C1D6666E2
:105730006626251C662626262E1C1D266666252521
:105740001C66666625251C6666661C1D6626262662
:105750006666262666666626266666662626666669
:105760001D01666666660A016666261400006626E6
:10577000261301002626660A01016666661D1401CD
:1057800066662626661D66262666666600005C013D
:105790000000000AFF0101000A13130A01000000C3
:1057A00000000000010A130A0101010101010101C9
:1057B0001D1D1D1D1D1D662626666666001D66666E
:1057C0006666000A66262626000014266626000164
:1057D0001366666601010A66666601141D262626A2
:1057E0001D6626266626662626666666FF37B73756
:1057F0006F14FF37B7376F14FF37B7376F14FF37A2
:10580000B7376F14FF37B7376F14FF37B7376F14D9
:10581000FF37B7376F14FF37B7376F14FF37B73716
:105820006F14FF37B7376F14FF2E1C376F14FF1C30
:105830000B376F14FF2E0B376F14FF2E0B376F14BF
:10584000FF1414146F14FF37B7376F14FF37B737CF
:105850006F14FF37B7376F14FF1C1C2E6F14FF3700
:10586000B71C6F14FF250B2E6F14FF1CB7376F1476
:10587000FF1414146F14FF37B7376F14FF37B7379F
:105880006F14FF37B7376F14FF1D14146F14FF37F1
:10589000B7136F14FF370B2E6F14FF37B71C6F143D
:1058A000FF1D1C2E6F14FF37B7376F14FF37B73744
:1058B0006F14FF37B7376F14FF14B7146F14FF134B
:1058C000B7136F14FF1C0B0B6F14FF37B70B6F145C
:1058D000FF37B7146F14FF37B7376F14FF37B73779
:1058E0006F14FF37B7376F14FF14141C6F14FF13B6
:1058F000B7376F14FF0B0B2E6F14FF37B71C6F14E5
:10590000FF141C2E6F14FF37B7376F14FF37B737EC
:105910006F14FF37B7376F14FF2E1C1D6F14FF1C59
:10592000B7376F14FF0B0B256F14FF0BB70B6F14FA
:10593000FF2513256F14FF37B7376F14FF37B737BD
:105940006F14FF37B7376F14FF1414146F14FF3739
:10595000AF1C6F14FF37652E6F14FF371C376F14A1
:10596000FF3714376F14FF37B7376F14FF37B73768
:105970006F14FF2E1C2E6F14FF0BB70B6F14FF1D3F
:10598000141D6F14FF0BB70B6F14FF0BAF0B6F14CD
:10599000FF2E1C2E6F14FF37B7376F14FFFFFFFF6A
:1059A000FFFFFF3737373737FF37B7B7B7B7FF379F
:1059B000B7373737FF37B7373737FF37B737373767
:1059C000FF37B7376F6FFF37B7376F14FFFFFFFF32
:1059D000FFFF373737376F14B7B7B7376F1437371D
:1059E000B7376F143737B7376F143737B7376F1488
:1059F0006F37B7376F14BF37B7376F14FF37B73705
:105A00006F14FF37B7373737FF37B7B7B7B7FF3739
:105A100037373737FF3737373737FF373737373786
:105A2000FF6F6F6F6F6FFF1414141414BF37B73705
:105A30006F143737B7376F14B7B7B7376F143737B7
:105A400037376F14373737376F14373737376F14A7
:105A50006F6F6F6F6F14141414141414B7B7777733
:105A6000B7B7B77777B7B7B77777B7B7B777B7B706
:105A7000B7777777B7B77777B7B7B77777B7B7B776
:105A80007777B7B7B777B7B7B777777726266666EA
:105A90006626666666262626666626266666662666
:105AA00026666666262666666666666666662626D6
:105AB000666626266666662626666666C0C0C0C01E
:105AC000C0C0C0C0C0C0C0C0C0C0C0C0C0C0C0C0D6
:105AD000C0C0C0C0C0C0C0C0C0C0C0C0C0C0C0C0C6
:105AE000C0C0C0C0C0C0C0C0C0C0C0C00000FFFFB8
:105AF000FF0000FF000000FF00FF0000FFFF00FFAD
:105B000000FF00FF00FFFF0000FF00FF000000FF9C
:105B10000000FFFFFF00000000000000000000FF89
:105B200000000000FFFF0000000000FF0000000078
:105B300000FF0000000000FF0000000000FF000068
:105B40000000FFFFFF000000000000000000FFFF5A
:105B5000FF0000FF000000FF0000000000FF000049
:105B600000FFFF000000FF00000000FF0000000039
:105B700000FFFFFFFFFF0000000000000000FFFF2C
:105B8000FF0000FF000000FF0000000000FF000019
:105B9000FFFFFF000000000000FF00FF000000FF0B
:105BA0000000FFFFFF0000000000000000000000F8
:105BB000FF00000000FFFF000000FF00FF0000FFEB
:105BC0000000FF0000FFFFFFFFFF00000000FF00DC
:105BD00000000000FF0000000000000000FFFFFFC9
:105BE000FFFF00FF0000000000FF0000000000FFBA
:105BF000FFFFFF000000000000FF00FF000000FFAB
:105C00000000FFFFFF00000000000000000000FF98
:105C1000FF000000FF00000000FF0000000000FF88
:105C2000FFFFFF0000FF000000FF00FF000000FF7B
:105C30000000FFFFFF0000000000000000FFFFFF6A
:105C4000FFFF0000000000FF00000000FF00000058
:105C500000FF00000000FF0000000000FF00000047
:105C60000000FF0000000000000000000000FFFF37
:105C7000FF0000FF000000FF00FF000000FF000029
:105C8000FFFFFF0000FF000000FF00FF000000FF1B
:105C90000000FFFFFF000000000000000000FFFF09
:105CA000FF0000FF000000FF00FF000000FF0000F9
:105CB000FFFFFFFF0000000000FF00000000FF00EA
:105CC0000000FFFF00000000000000000000FFFFD8
:105CD000FF0000FF000000FF00FF000000FF00FFCA
:105CE000000000FF00FFFFFFFFFF00FF000000FFBC
:105CF00000FF000000FF00000000000000FFFFFFA9
:105D0000FF0000FF000000FF00FF000000FF00FF99
:105D1000FFFFFF0000FF000000FF00FF000000FF8A
:105D200000FFFFFFFF000000000000000000FFFF79
:105D3000FF0000FF000000FF00FF0000000000FF68
:105D40000000000000FF0000000000FF000000FF56
:105D50000000FFFFFF0000000000000000FFFFFF49
:105D6000FF0000FF000000FF00FF000000FF00FF39
:105D7000000000FF00FF000000FF00FF000000FF28
:105D800000FFFFFFFF0000000000000000FFFFFF1A
:105D9000FFFF00FF0000000000FF0000000000FF08
:105DA000FFFFFF0000FF0000000000FF00000000F8
:105DB00000FFFFFFFFFF00000000000000FFFFFFEB
:105DC000FFFF00FF0000000000FF0000000000FFD8
:105DD000FFFFFF0000FF0000000000FF00000000C8
:105DE00000FF000000000000000000000000FFFFB6
:105DF000FF0000FF000000FF00FF0000000000FFA8
:105E000000FFFFFF00FF000000FF00FF000000FF99
:105E10000000FFFFFFFF00000000000000FF000087
:105E200000FF00FF000000FF00FF000000FF00FF78
:105E3000FFFFFFFF00FF000000FF00FF000000FF6A
:105E400000FF000000FF000000000000000000FF55
:105E5000000000FFFFFFFFFF0000FFFFFF0000004A
:105E600000FF0000000000FF00000000FFFFFF0037
:105E700000FFFFFFFFFF0000000000000000FFFF29
:105E8000000000FFFFFFFF0000FF00FFFF00000019
:105E900000FFFF000000FFFFFF000000FFFFFF000A
:105EA00000FFFFFFFFFF00000000000000FF00FFF9
:105EB00000FF00FFFFFFFFFF0000FFFFFF000000EB
:105EC000FFFFFF000000FFFFFF000000FFFFFF00DB
:105ED00000FFFFFFFFFF000000000000000000FFC8
:105EE0000000000000FF00000000FFFFFF0000FFB7
:105EF000FFFFFFFF0000FFFFFF000000FFFFFF00AC
:105F000000FFFFFFFFFF000000000000000000FF97
:105F10000000000000FF0000000000FF000000FF84
:105F2000FFFFFFFF000000FF0000000000FF000077
:105F3000000000FF000000000000000000FF000063
:105F400000FF00FF0000FF00000000FF0000000055
:105F5000FF00000000FF0000FFFF0000000000FF46
:105F600000000000FF0000000000FFFF00FF000035
:105F700000FF00FFFF00FFFF00FF00FF00FF00FF2A
:105F8000000000FF00FF000000FF00FF000000FF16
:105F900000FF000000FF0000000000000000FFFF05
:105FA000FF0000FF000000FF00FF000000FF00FFF7
:105FB000000000FF00FF000000FF00FF000000FFE6
:105FC0000000FFFFFF00000000000000C7C7C7C7B8
:105FD000C7C7C7C7C7C7C7C7C7C7C7C7C7C7C7C751
:105FE000C7C7C7C7C7C7C7C7C7C7C7C7C7C7C7C741
:105FF000C7C7C7C7C7C7C7C7C7C7C7C7281C000009
:106000000000000000000000000000000000000090
:106010000000000000000000000000000000000080
:106020000000000000000000A78F908F8F918F8FDD
:10603000928F8F938F8F948F8F958F8F968F8F974F
:106040008FA8000000000000000000000000000019
:106050009EABABABACACACABABABACACACABABAB97
:10606000ACACACABABABACACAC9E00000000000089
:106070000000000000000000A6ABABABACACACABCA
:10608000ABABACACACABABABACACACABABABACAC58
:10609000ACA60000000000000000000000000000AE
:1060A0009EABABABACACACABABABACACACABABAB47
:1060B000ACACACABABABACACAC9E00000000000039
:1060C00000000000000000009EACACACABABABAC81
:1060D000ACACABABABACACACABABABACACACABAB08
:1060E000AB9E000000000000000000000000000067
:1060F000A5ACACACABABABACACACABABABACACACED
:10610000ABABABACACACABABABA5000000000000E4
:1061100000000000000000009EACACACABABABAC30
:10612000ACACABABABACACACABABABACACACABABB7
:10613000AB9E000000000000000000000000000016
:106140009EABABABACACACABABABACACACABABABA6
:10615000ACACACABABABACACAC9E00000000000098
:106160000000000000000000A4ABABABACACACABDB
:10617000ABABACACACABABABACACACABABABACAC67
:10618000ACA40000000000000000000000000000BF
:106190009EABABABACACACABABABACACACABABAB56
:1061A000ACACACABABABACACAC9E00000000000048
:1061B00000000000000000009EACACACABABABAC90
:1061C000ACACABABABACACACABABABACACACABAB17
:1061D000AB9E000000000000000000000000000076
:1061E000A3ACACACABABABACACACABABABACACACFE
:1061F000ABABABACACACABABABA3000000000000F6
:1062000000000000000000009EACACACABABABAC3F
:10621000ACACABABABACACACABABABACACACABABC6
:10622000AB9E000000000000000000000000000025
:106230009EABABABACACACABABABACACACABABABB5
:10624000ACACACABABABACACAC9E000000000000A7
:106250000000000000000000A2ABABABACACACABEC
:10626000ABABACACACABABABACACACABABABACAC76
:10627000ACA20000000000000000000000000000D0
:106280009EABABABACACACABABABACACACABABAB65
:10629000ACACACABABABACACAC9E00000000000057
:1062A00000000000000000009EACACACABABABAC9F
:1062B000ACACABABABACACACABABABACACACABAB26
:1062C000AB9E000000000000000000000000000085
:1062D000A1ACACACABABABACACACABABABACACAC0F
:1062E000ABABABACACACABABABA100000000000007
:1062F00000000000000000009EACACACABABABAC4F
:10630000ACACABABABACACACABABABACACACABABD5
:10631000AB9E000000000000000000000000000034
:106320009EABABABACACACABABABACACACABABABC4
:10633000ACACACABABABACACAC9E000000000000B6
:106340000000000000000000A0ABABABACACACABFD
:10635000ABABACACACABABABACACACABABABACAC85
:10636000ACA00000000000000000000000000000E1
:106370009EABABABACACACABABABACACACABABAB74
:10638000ACACACABABABACACAC9E00000000000066
:1063900000000000000000009EACACACABABABACAE
:1063A000ACACABABABACACACABABABACACACABAB35
:1063B000AB9E000000000000000000000000000094
:1063C0009FACACACABABABACACACABABABACACAC20
:1063D000ABABABACACACABABAB9F00000000000018
:1063E00000000000000000009EACACACABABABAC5E
:1063F000ACACABABABACACACABABABACACACABABE5
:10640000AB9E000000000000000000000000000043
:10641000A98F908F8F918F8F928F8F938F8F948F63
:106420008F958F8F968F8F978FAA000000000000A6
:10643000000000000000000000000000000000005C
:10644000000000000000000000000000000000004C
:106450000000000000000000000000000000280212
:10646000000000000000000000000000000000002C
:10647000000000000000000000000000000000001C
:1064800000000000000000000000A78F908F8F9197
:106490008F8F928F8F938F8F948F8F958F8F968FF3
:1064A0008F978FA80000000000000000000000008F
:1064B0000E05A78F8F8F8F8F8F8F8F8F8F8F8FA8C6
:1064C0009EABABABACACACABABABACACAC9E9EAB3D
:1064D000ABABACACACABABABACACAC9E9EABABAB20
:1064E000ACACACABABABACACAC9EA98F8F8F8F8F91
:1064F0008F8F8F8F8F8F8FAA0002060000CE00FF34
:106500000000EC0001020107000207FF0001030088
:10651000FF0002080007E00000EC0008500204063B
:1065200002040602050000FF0002050007A00008A3
:106530002305050000FF0002040007D000083C000E
:106540000990000A3C020306020306010306010348
:106550000601030601050000FF0002050007A00078
:1065600008280507400207A005050000FF0000FB02
:106570000002080009A0000A3200084600FF0002DD
:10658000040007A00000F600083201030101030126
:106590000103010103010103010508280007FF00B1
:1065A00002010000F60009A0000A3200FF00020804
:1065B00000000A00072000083205084105084605CA
:1065C000084B07084105084605084B05084D00091A
:1065D000A0000A320000F600FF0002000000FB00ED
:1065E000084802030201030201030201030201033E
:1065F0000202040A01030201030201030201030271
:106600000103020204020103020103020103020169
:10661000030201030202040A01030201030201034F
:106620000201030201030202040501030201030245
:106630000103020103020103020204050103020136
:10664000030201030201030201030201050000FF2E
:1066500000020300085602040A02040802040602AB
:1066600004040204020008420203050204020203B9
:10667000050203050204020203050000F8040305F5
:1066800004040504030504040504030504040504C7
:10669000030501050000FF0002060000FB00FF00EB
:1066A0000000F86400000000000000F86400000032
:1066B00000000000F86400000000000000F8640022
:1066C000000000010000F86400000000000000F875
:1066D0006400000000000000F864000000000100F9
:1066E00000F86400000000000000F86400000000F2
:1066F000010000F86400000000010000F8640000E0
:106700000000000000F86400000000000000F864D1
:1067100000000000000000F864000000000100001C
:10672000F86400000000010000F8640000000000B0
:106730000000F86400000000000000006500000098
:1067400000000000F86400000000000000F8640091
:10675000000000000000F86400000000000000F8E5
:106760006400000000000000F86400000000000069
:1067700000F86400000000000000F8640000000061
:10678000000000F86400000000000000F864000051
:106790000000000000F86400000000000000F86441
:1067A00000000000000000F864000000000000008D
:1067B000F864000000000000001165000000000007
:1067C00000002865000000000000003665000000A1
:1067D000000000005965000000000000006D650029
:1067E0000000000000007E6500000000000000AD19
:1067F0006500000000000000D965000000000000F6
:1068000000506600000000000000976600000000D5
:1068100000C01100B0077F00C10300B1077F00C2B4
:106820000B00B2077F0092326900C30700B3077FF5
:1068300000930D3200903E7F0A9232690093073E2A
:1068400002903E7F049232690093073E01903E7FA2
:1068500005922D690093073E0190397F0B922D69B7
:106860000093073E0090397F0B92326900930D32FE
:1068700001903E7F0B9232690093073E01903E7F6C
:10688000049232690093073E01903E7F05922D6984
:106890000093073E0190397F0B922D690093073ECC
:1068A0000190397F0A92326900930D3201903E7F48
:1068B0000A9232690093073E01903E7F0592326949
:1068C0000093073E01903E7F05922D690093073E9D
:1068D0000190397F0A922D690093073E0190397F1C
:1068E0000B92326900930D3201903E7F0A92326919
:1068F0000093073E01903E7F059232690093073E68
:1069000001903E7F05922D6900930D320190397FF1
:106910000B922D6900930D370090397F0BFF060114
:10692000530092326900930D3C01903E7F009139F3
:106930005D0A9232690093073E0190457F009141C4
:106940005D059232690093073E06922D6900930718
:106950003E00904A7F0091415D0B922D69009307A4
:106960003E0190497F0091435D0B9232690093078D
:106970003E01904A7F0091415D0A9232690093077F
:106980003E0190457F0091405D059232690093077A
:106990003E0190457F0091415D05922D690093076E
:1069A0003E0190467F0091435D0A922D6900930756
:1069B0003E0190437F0091405D0B92326900930746
:1069C0003E0090457F0091415D0B92326900930734
:1069D0003E0190417F00913D5D0592326900930731
:1069E0003E0090417F00913E5D05922D6900930726
:1069F0003E0190437F0091405D0B922D690093070B
:106A00003E0190407F00913D5D0A923269009307FC
:106A10003E0190417F00913E5D0B923269009307E9
:106A20003E01903E7F0091385D05923269009307E8
:106A30003E01903E7F0091395D05922D69009307DC
:106A40003E0090407F00913D5D0B922D69009307C1
:106A50003E01903D7F0091395D0A923269009307B3
:106A60003E01903E7F0091395D0B923269009307A1
:106A70003E0090397F0091355D05923269009307A1
:106A80003E069231690093073E01903A7F009137AC
:106A90005D0B922D690093073E01903D7F00913779
:106AA0005D0A9232690093073E01903E7F00913962
:106AB0005D0B9232690093073E0190397F0091355A
:106AC0005D059232690093073E0592316900930794
:106AD0003E01903A7F0091375D0B922D690093073C
:106AE0003E0190407F00913D5D0A9232690093071C
:106AF0003E01903E7F0091395D0A92326900930712
:106B00003E0190457F0091415D05923269009307F7
:106B10003E06922D690093073E01904A7F00914105
:106B20005D0A922D690093073E0190497F009143D1
:106B30005D0B9232690093073E01904A7F009141BC
:106B40005D0B9232690093073E0090457F009140B3
:106B50005D059232690093073E0190457F009141A7
:106B60005D05922D690093073E0190467F00914399
:106B70005D0A922D690093073E0290437F00914089
:106B80005D0A9232690093073E0190457F00914172
:106B90005D0A9232690093073E0190417F00913D6A
:106BA0005D059232690093073E0190417F00913E5E
:106BB0005D05922D690093073E0190437F0091404F
:106BC0005D0A922D690093073E0190407F00913D40
:106BD0005D0B9232690093073E0190417F00913E28
:106BE0005D0A9232690093073E01903E7F00913822
:106BF0005D059232690093073E01903E7F00913916
:106C00005D05922D690093073E0190407F00913D04
:106C10005D0A922D690093073E01903D7F009139F6
:106C20005D0A9232690093073E02903E7F009139DF
:106C30005D0A9232690093073E0190397F009135D9
:106C40005D059232690093073E0692316900930711
:106C50003E00903A7F0091375D0B922D69009307BB
:106C60003E01903D7F0091375D0B923269009307A2
:106C70003E00903E7F0091395D0B92326900930790
:106C80003E0190397F0091355D059232690093078E
:106C90003E059231690093073E02903A7F0091379A
:106CA0005D0A922D690093073E0190407F00913D5F
:106CB0005D0A9232690093073E01903E7F00913950
:106CC0005D0B9232690093073E069232690093078A
:106CD0003E05922E690093073E0C922B69009307A4
:106CE0003E0B9232690093073E0C92326900930783
:106CF0003E059232690093073E0692316900930780
:106D00003E0190407F0091395D0A922D6900930702
:106D10003E02903D7F0091395D0A923269009307EF
:106D20003E01903E7F0091395D0B923269009307DE
:106D30003E059232690093073E06922E6900930742
:106D40003E0C922B690093073E0B92326900930729
:106D50003E0B9232690093073E0692326900930718
:106D60003E06922B690093073E0190407F00913CC4
:106D70005D0A9224690C29690093073E0190417FC6
:106D80000A9235690093073E0190417F0592296977
:106D90000093073E0190417F059224690093073ECE
:106DA0000190437F0A9230690093073E0190407F33
:106DB0000B9229690093073E0190417F0A92356941
:106DC0000093073E0190417F059229690093073E99
:106DD0000190417F049224690093073E0290437F13
:106DE0000A9230690093073E0190407F0B92296917
:106DF0000093073E0090417F0B9235690093073E58
:106E0000069229690093073E069224690093073E83
:106E10000B9230690093073E0B9229690093073E5D
:106E20000C9235690093073E059229690093073E4D
:106E3000069224690093073E0190437F0091405DD4
:106E40000B9230690093073E0B9229690093073E2D
:106E50000190457F0091415D0B9235690093073E9B
:106E60000190457F0091415D059229690093073E9D
:106E70000190457F0091415D049224690093073E93
:106E80000190467F0091435D0B9230690093073E6D
:106E90000190437F0091405D0A9229690093073E6B
:106EA0000190457F0091415D0A9235690093073E4C
:106EB0000290457F0091415D049229690093073E4D
:106EC0000190457F0091415D059224690093073E42
:106ED0000190467F0091435D0B9230690093073E1D
:106EE0000090437F0091405D0B9229690093073E1B
:106EF0000190457F00913C5D0B9235690093073E00
:106F0000059229690093073E069224690093073E83
:106F10000C9230690093073E0B9229690093073E5B
:106F20000B9235690093073E069229690093073E4C
:106F300006922B690093073E0190477F00913E5DCA
:106F40000A9237690093073E0C9224690093073E2A
:106F50000190487F0091405D0A9230690093073E9E
:106F60000190487F0091415D059224690093073E9E
:106F70000190487F0091435D059224690093073E8C
:106F80000190487F0091405D0B9230690093073E6D
:106F90000090487F0091435D0B9229690093073E62
:106FA00001904A7F0091455D0A9235690093073E42
:106FB0000190487F0091455D059229690093073E45
:106FC000069229690093073E0090487F0091455D35
:106FD0000B9235690093073E0190477F00913E5D1B
:106FE0000B9224690093073E0190487F0091405D19
:106FF0000A9230690093073E0190487F0091415DFD
:10700000059224690093073E0190487F0091435DFB
:10701000059224690093073E0190487F0091405DEE
:107020000A9230690093073E0190487F0091435DCA
:107030000B9229690093073E00904A7F0091445DBE
:107040000B9235690093073E0190487F0091445DA3
:10705000059229690093073E059229690093073E2E
:107060000190487F0091445D0B9235690093073E83
:107070000190477F00913E5D0A9224690093073E8C
:107080000190487F0091405D0B9230690093073E6C
:107090000190487F0091415D059224690093073E6D
:1070A0000190487F0091435D059224690093073E5B
:1070B0000090487F0091405D0B9230690093073E3D
:1070C0000190487F0091435D0A9224690093073E36
:1070D0000190477F00913E5D0B9230690093073E1F
:1070E0000090477F0091405D059224690093073E20
:1070F0000190477F0091415D059224690093073E0E
:107100000190477F00913E5D0B9230690093073EEE
:107110000190477F0091415D0A9224690093073EE8
:107120000190467F00913E5D0B9230690093073ECF
:107130000190467F0091405D059224690093073ECF
:107140000090467F0091415D059224690093073EBF
:107150000190467F0091405D0B9230690093073E9D
:107160000190437F0091405D0A9224690093073E9D
:107170000190407F0091375D0A9230690093073E8D
:107180000190417F00913E5D059224690093073E86
:10719000069224690093073E0190437F0091405D71
:1071A0000A9230690093073E01903C7F0091345D64
:1071B0000B9226690093073E0190437F0091395D51
:1071C0000B9232690093073E0090417F0091395D38
:1071D000059226690093073E0190417F0091395D39
:1071E000059226690093073E01903C7F0091395D2E
:1071F0000A9232690093073E0290417F0091395D07
:107200000A9226690B32690093073E01903C7F0089
:1072100091395D059226690093073E01903E7F00FB
:10722000913B5D059226690093073E01903C7F00EB
:1072300091395D0A9232690093073E0190397F00CF
:1072400091355D0B9226690093073E0190437F00C4
:1072500091385D0A9232690093073E0190417F00A8
:1072600091385D059226690093073E0190417F00A9
:1072700091385D059226690093073E01903C7F009E
:1072800091385D0A9232690093073E0190417F0078
:1072900091385D0A9226690C32690093073E01908D
:1072A0003C7F0091385D059226690093073E01906E
:1072B0003E7F00913A5D049226690093073E01905B
:1072C0003C7F0091385D0B9232690093073E01903C
:1072D000387F0091355D0B9224690093073E009042
:1072E0003C7F0091345D0B9230690093073E06921B
:1072F00024690093073E059224690093073E0C928F
:1073000030690093073E0B9224690093073E0C926C
:1073100030690093073E069224690093073E059268
:1073200024690093073E0C9230690093073E0B924C
:1073300024690093073E0C9230690093073E059242
:1073400024690093073E069224690093073E0B923E
:1073500030690093073E0C9224690093073E0C921B
:1073600030690093073E059224690093073E069218
:1073700034690093073E01903D7F0091375D16927E
:1073800032690093073E01903E7F0A923269009372
:10739000073E02903E7F049232690093073E0190BF
:1073A0003E7F05922D690093073E0190397F0A9236
:1073B0002D690093073E0190397F0B92326900934B
:1073C000073E01903E7F0A9232690093073E01908A
:1073D0003E7F059232690093073E01903E7F059201
:1073E0002D690093073E0190397F0A922D69009321
:1073F000073E0190397F0B9232690093073E01905E
:107400003E7F0A9232690093073E01903E7F0592CB
:1074100032690093073E01903E7F04922D690093EC
:10742000073E0290397F0A922D690093073E019032
:10743000397F0B9232690093073E00903E7F0B929A
:1074400032690093073E01903E7F059232690093B6
:10745000073E01903E7F05922D690093073E009004
:10746000397F0B922D690093073E0190397F0AFF07
:10747000060145009232690093073E02903E7F006C
:1074800091395D0A9232690093073E0190457F0071
:1074900091415D049232690093073E06922D690086
:1074A00093073E01904A7F0091415D0B922D690048
:1074B00093073E0190497F0091435D0A9232690033
:1074C00093073E01904A7F0091415D0B9232690023
:1074D00093073E0190457F0091405D05923269001F
:1074E00093073E0190457F0091415D04922D690014
:1074F00093073E0190467F0091435D0B922D6900FA
:1075000093073E0190437F0091405D0A92326900EB
:1075100093073E0190457F0091415D0A92326900D8
:1075200093073E0290417F00913D5D0492326900D5
:1075300093073E0190417F00913E5D05922D6900C9
:1075400093073E0190437F0091405D0B922D6900AF
:1075500093073E0090407F00913D5D0B92326900A1
:1075600093073E0190417F00913E5D0B923269008E
:1075700093073E01903E7F0091385D04923269008E
:1075800093073E01903E7F0091395D05922D690081
:1075900093073E0190407F00913D5D0B922D690065
:1075A00093073E01903D7F0091395D0A9232690058
:1075B00093073E01903E7F0091395D0A9232690047
:1075C00093073E0190397F0091355D059232690045
:1075D00093073E069231690093073E01903A7F007F
:1075E00091375D0A922D690093073E01903D7F001F
:1075F00091375D0B9232690093073E01903E7F0008
:1076000091395D0A9232690093073E0190397F00FB
:1076100091355D059232690093073E06923169000B
:1076200093073E01903A7F0091375D0B922D6900E0
:1076300093073E0090407F00913D5D0B92326900C0
:1076400093073E01903E7F0091395D0A92326900B6
:1076500093073E0190457F0091415D05923269009C
:1076600093073E06922D690093073E00904A7F00E3
:1076700091415D0B922D690093073E0190497F0077
:1076800091435D0B9232690093073E01904A7F005F
:1076900091415D0A9232690093073E0190457F0057
:1076A00091405D059232690093073E0190457F004D
:1076B00091415D05922D690093073E0190467F0040
:1076C00091435D0A922D690093073E0190437F002C
:1076D00091405D0B9232690093073E0090457F0018
:1076E00091415D0B9232690093073E0190417F000A
:1076F000913D5D059232690093073E0090417F0005
:10770000913E5D05922D690093073E0190437F00F5
:1077100091405D0B922D690093073E0190407F00E0
:10772000913D5D0A9232690093073E0190417F00CE
:10773000913E5D0B9232690093073E01903E7F00BF
:1077400091385D059232690093073E01903E7F00BB
:1077500091395D05922D690093073E0090407F00AE
:10776000913D5D0B922D690093073E01903D7F0096
:1077700091395D0A9232690093073E01903E7F0085
:1077800091395D0B9232690093073E0090397F007A
:1077900091355D059232690093073E06923169008A
:1077A00093073E01903A7F0091375D0B922D69005F
:1077B00093073E01903D7F0091375D0A9232690048
:1077C00093073E01903E7F0091395D0B9232690034
:1077D00093073E0190397F0091355D059232690033
:1077E00093073E059231690093073E01903A7F006E
:1077F00091375D0B922D690093073E0190407F0009
:10780000913D5D0A9232690093073E01903E7F00F0
:1078100091395D0A9232690093073E0692326900FF
:1078200093073E06922E690093073E0B922B690048
:1078300093073E0C9232690093073E0C9232690026
:1078400093073E059232690093073E069231690024
:1078500093073E0190407F0091395D0A922D6900A7
:1078600093073E02903D7F0091395D0A9232690094
:1078700093073E01903E7F0091395D0A9232690084
:1078800093073E069232690093073E06922E6900E6
:1078900093073E0B922B690093073E0C92326900CE
:1078A00093073E0B9232690093073E0692326900BD
:1078B00093073E06922B690093073E0190407F009C
:1078C000913C5D0A9224690B29690093073E01905F
:1078D000417F0B9235690093073E0190417F0592ED
:1078E00029690093073E0190417F04922469009327
:1078F000073E0190437F0B9230690093073E019051
:10790000407F0B9229690093073E0090417F0B92C4
:1079100035690093073E0190417F059229690093E4
:10792000073E0190417F049224690093073E029034
:10793000437F0A9230690093073E0190407F0A928C
:1079400029690093073E0190417F0B9235690093AE
:10795000073E069229690093073E05922469009329
:10796000073E0C9230690093073E0B922969009301
:10797000073E0C9235690093073E059229690093F2
:10798000073E069224690093073E0190437F0A92C6
:1079900030690093073E0C9229690093073E0190DD
:1079A000457F0B9235690093073E0090457F059215
:1079B00029690093073E0190457F05922469009351
:1079C000073E0190467F0B9230690093073E00907E
:1079D000437F0B9229690093073E0190457F0A92ED
:1079E00035690093073E0290457F04922969009310
:1079F000073E0190457F059224690093073E019060
:107A0000467F0A9230690093073E0190437F0AFF48
:107A10002F000303ABABABABABABABABAB03030127
:107A200002031011121F202103030405061314156D
:107A3000222324030307080916171822232403030B
:107A40000A0B0C191A1B22232403030D0E0F1C1DF5
:107A50001E22232403032526271C1D1E2223240364
:107A600003ACACACACACACACACAC03032E2F303D37
:107A7000113E98999A03033132333F14402B2C2D39
:107A800003033435364142432B2C2D030337383959
:107A9000441A452B2C2D03033A3B3C461D472B2C07
:107AA0002D030328292A461D472B2C2D0303ABAB9E
:107AB000ABABABABABABAB030348494A57585966CA
:107AC000676803034B4C4D5A5B5C696A6B03034E5A
:107AD0004F505D5E5F696A6B030351525360616290
:107AE000696A6B0303545556636465696A6B0303E3
:107AF0006C6D6E636465696A6B0303ACACACACAC73
:107B0000ACACACAC03037576778458859B9C9D0325
:107B10000378797A865B879B9C9D03037B7C7D88B9
:107B2000898A9B9C9D03037E7F808B618C9B9C9D9F
:107B300003038182838D648E9B9C9D03036F707110
:107B40008D648E9B9C9D0303ADADADADADADADAD74
:107B5000AD48756D616E20286A6F7970616420315F
:107B6000290048756D616E20286A6F797061642004
:107B7000322900435055202865617379290000009F
:107B80000000000043505520286D656469756D291B
:107B900000000000004350552028686172642900ED
:107BA000000000000000435055202865787472657D
:107BB0006D6529000000004E6F000059657300429A
:107BC0006C61636B3A0057686974653A00536F756E
:107BD0006E643A004D757369633A00547572626F52
:107BE0003A00707265737320535441525420746F7D
:107BF00020706C6179003E0011241FBECFEFD0E1F0
:107C0000DEBFCDBF11E0A0E0B1E0E8E8F9EB02C0D3
:107C100005900D92A230B107D9F728E0A2E0B1E0BB
:107C200001C01D92A23FB207E1F714BE0FB6F8944F
:107C3000A895809160008861809360001092600038
:107C40000FBEF8948EE990E0FC0125913491F90182
:107C5000FF273083029620E0803D9207A9F70E941B
:107C6000A641811102C00E948441EBE7F5E080E863
:107C7000819397E0E738F907D9F78BE795E0909380
:107C80008807809387071092890710928C071092BB
:107C900092071092980710929E0710926605109214
:107CA000680582E18093670580EE80936E0584E12C
:107CB00080936D05109272051092710510927605F1
:107CC0001092750581E080938B070E94374D789460
:107CD0000E94004D0E94075C0C94C25C0C94000052
:107CE000E0E0EA95F1F7E1ECEA95F1F7C2E0D1E0E6
:107CF000A0906E05662776E035D13AE23A95F1F725
:107D00000E94A83E30E13A95F1F7AA9489F0C8950F
:107D10006395683029F0C895C895C8950000ECCFE8
:107D20006627002438E2C30FD01DC8950000E4CFB9
:107D300035E03A95F1F700C015D1E091680542E0D1
:107D4000E160E427E0936805E2E0E09336000895FF
:107D5000DE0110E38091620590916305679F800DBD
:107D6000911D4D91419F080E191EF00128E20591C9
:107D700008B94D91059108B9419F059108B9AC0129
:107D8000400D059108B9511D0000059108B90591F4
:107D9000FA012A9508B959F700C00000002708B970
:107DA00008950F921F92EF93FF93FFB7E091840025
:107DB000FF93E2FD04C0E1FD02C0000000C0E0FF4F
:107DC00000C0E0916705EA95E0936705F0916605CC
:107DD000F0FD51C0EC3098F0F3E0F0938900FDE83D
:107DE000F0938800E0FB289826F4E1E00E94AC4084
:107DF000B2C0E5E1EA95F1F70000289AACC0E630A0
:107E000008F100C000C02898E0FBE4E016F40E94EE
:107E1000AC40E4E0E0933600E6E0E0936F009BC006
:107E2000EF93E0918400E2FD04C0E1FD02C0000098
:107E300000C0E0FF00C0E2E00000289AE0936F007D
:107E4000EF91189500C0E0FB289826F4E1E00E942D
:107E5000AC4005C0E5E1EA95F1F70000289AE09111
:107E60006705E03009F077C0EDEFE0936705E1E0EA
:107E7000E093660570C0E7E0E0938900EBE1E093F2
:107E8000880000C02898E2E000C00E94AC40FDEFEE
:107E900000906D05F019E0916705EF17D8F4FDEF3C
:107EA00000906D05F01900906E05F019EF1790F035
:107EB000EDE1FF2700800F92EA95E1F70FE10A95C7
:107EC000F1F700C00E94703EE1E0FF270F900192A1
:107ED000EE31E0F3E0916705E03009F03CC02F930C
:107EE0003F934F935F936F937F938F939F93AF9342
:107EF000BF9378941124EE27E0936605E2E1E093C6
:107F000067058091770590917805019680937705B4
:107F100090937805E0916905F0916A05E115F10506
:107F200009F009950E9474410E94384D0E94BD3F9E
:107F30001124E0916B05F0916C05E115F10509F054
:107F40000995BF91AF919F918F917F916F915F91B3
:107F50004F913F912F91EF91EFBFFF91EF911F90C4
:107F60000F9018952898E2E000C00E94AC40E09184
:107F70006705EA95E09367050895E0918B07E0FDBA
:107F80000E948C4300908907002019F4ABE7B5E00C
:107F900002C0A1E8B6E021E002260092890722E0B3
:107FA00020938A07E0918B07E0FF08952F923F927C
:107FB0004F925F926F927F928F929F92AF92BF92F9
:107FC000CF92DF92EF92FF920F931F93CF93DF93A5
:107FD00050919E07E091A207F091A3078091A1071D
:107FE00040909F075090A00766245F010090A4076F
:107FF0001090A507A018B1088090A6079090A70739
:108000001D01C3E8840DE51DF61DE815F90508F00E
:10801000F501449145031D92840DE51DF61DE815FB
:10802000F90508F0F501449145031D92CA9551F7F1
:10803000D10150939E07E093A207F093A30780938A
:10804000A10720908D0730908E07409090075090A8
:10805000910760908F0710918C0770909307809024
:10806000940790909507A0909607B090970720915D
:108070009207C0909907D0909A07E0909C07F090E3
:108080009D0700919B07309198079FEFCC91DD27CA
:10809000C7FDDFEF620C431CF2014491410300086D
:1080A000C10DD01D970CA81CF50144914203000896
:1080B000C10DD01D0C0DED1CF701449143030008C8
:1080C000C10DD01D0024C038D0050CF0CFE70A94B4
:1080D000C038D0050CF4C0E8C058CD939A9509F08B
:1080E000D5CF40918A074A9540938A0797E009F0D7
:1080F000CDCF60928F074092900790929507A09203
:10810000960700939B07E0929C07DF91CF911F9108
:108110000F91FF90EF90DF90CF90BF90AF909F9026
:108120008F907F906F905F904F903F902F90089529
:10813000E0918707F0918807019100000093B30058
:1081400007E0E738F0070BE715E008F0F801E093E7
:108150008707F093880708950F931F932F93EF934A
:10816000E0918707F091880701910093B30007E041
:10817000E738F0070BE715E008F0F801E093870710
:10818000F0938807E8E0EA95F1F7EF912F911F91BE
:108190000F91E0FD289AE0FF01C00895F4E1FA95FF
:1081A000F1F700C0E1FD289AE1FF00C00895E0E684
:1081B000F4E0A2E0B1E01D923197E9F711240895AF
:1081C0009927772728E2629F080E191EA2E0B1E0E6
:1081D000A00DB11D4C9311240895992728E2629FA8
:1081E000080E191EA2E0B1E0A00DB11D509164056A
:1081F000450F4C931124089580936405089580934E
:1082000062059093630508958091680581700895D3
:10821000209168052E7F209368050895882329F40E
:1082200080916F05909170050895809173059091EC
:1082300074050895E0E6F0E0808183FD089588E10B
:1082400098E0F894808390837894FFCFF999FECFDB
:1082500092BD81BD60BDF894FA9AF99A7894089518
:10826000F999FECF92BD81BDF894F89A80B57894C3
:10827000089560936E0580936D050895129AC895D0
:10828000C895C895C895129840E180E090E020E03C
:1082900030E03695279596958795C895C895C895E9
:1082A000C8951398009B3068019B9068139AC895F5
:1082B000C895C895C895415061F7309370052093D3
:1082C0006F05909374058093730580916F0590916D
:1082D00070050F9731F080917305909174050F9799
:1082E00011F40C941A4108951092A807009903C044
:1082F00081E08093A807019905C08091A80782605A
:108300008093A8070C943E41CF93DF93C0E0D0E068
:10831000FE01E258FF4F6491CE010E942641219652
:10832000C032D105A9F7C0E2D0E06FEFCE010E94C4
:1083300026416FEFCE0101960E942641A096C115FD
:1083400088E0D80791F7DF91CF910895CF9380E02F
:1083500090E00E943041C82F81E090E00E943041BF
:10836000282F30E0322F22272C0F311D81E02A35B3
:10837000354509F080E0CF910895EF92FF920F9379
:108380001F93CF93DF9300D01F92CDB7DEB78C0140
:108390001A8219821B82AE014D5F5F4FBE016F5F73
:1083A0007F4FFC01808191810E943A42882311F025
:1083B000833019F589819A81892B49F48B8188232F
:1083C000D9F0F0E28F9FC00111249A83898378014C
:1083D00020E2E20EF11CF80161918F0189819A81FE
:1083E0009C012F5F3F4F3A8329830E9426410E153F
:1083F0001F0589F780E001C082E00F900F900F9079
:10840000DF91CF911F910F91FF90EF900895CF9240
:10841000DF92FF920F931F93CF93DF9300D0CDB7DE
:10842000DEB78B0140E050E0BE016F5F7F4F0E94DE
:108430003A42F82E811113C0680180E2C80ED11CA7
:1084400089819A819C012F5F3F4F3A8329830E9443
:108450003041F80181938F01EC15FD0589F78F2DCF
:108460000F900F90DF91CF911F910F91FF90DF90B0
:10847000CF9008958F929F92AF92BF92CF92DF924A
:10848000EF92FF920F931F93CF93DF93FB01118223
:1084900010828F3FFFEF9F0789F16A018B017C01FA
:1084A000A12CB12CC0E0D3E0912CC5010E94304139
:1084B000882EC50101960E943041282F30E0322FCE
:1084C0002227280D311D2E153F0529F4F801B18210
:1084D000A082D0E00BC02F3F3F4F41F4911006C067
:1084E000C114D10411F0F601C0839C2ECF5FF0E2DD
:1084F000AF0EB11CC034C9F68D2F01C081E0DF91F1
:10850000CF911F910F91FF90EF90DF90CF90BF9090
:10851000AF909F908F900895FC016787089508950C
:10852000FC0182810C94EF46FC019181690F61830B
:1085300082810C94DB46FC019181961B692F91830B
:1085400082810C94DB46FC0190819F759083089595
:10855000FC019081906490830895FC0166870895E2
:108560001F93CF93DF93EC01162F8A810E94DB4685
:1085700019838881877F8883DF91CF911F91089528
:10858000FC0162870895FC0163870895CF93DF9310
:10859000EC01462F298130E0F901EE0FFF1FE85F63
:1085A000F14765917491F901E40FF11D47FDFA95CA
:1085B000EE0FFF1FE85FF14785919491861B970BA3
:1085C000688570E00E94A85C6115710511F461E096
:1085D00070E0EA8186E0E89FF0011124E457F84F4B
:1085E00081819281860F971F928381837E836D8321
:1085F0008881886088838981480F4F83DF91CF917C
:108600000895FC0160870895FC0164830895DC01EE
:1086100014968C911497882319F155962D913C91BD
:108620005697662379F0062E000C770B6F5F7F4F0D
:10863000AB01440F551F640F751F261B370B09C074
:10864000EF3F39F023503109F9013297E491ED30D1
:10865000B9F756963C932E935597815014968C9368
:10866000089590930A08809309088FE680930C0878
:1086700010927A05EBEBF7E080E090E13FEF28E124
:10868000DF011E978C9312979C931D961C92119755
:108690003C93108211972C9313979C938F5F77963E
:1086A000843071F70895EBEAF7E03FEF20812F77F0
:1086B00020833383779628E0E730F207B9F70196F5
:1086C00090931108809310089093AA078093A907AC
:1086D000909313088093120810920E0810920D08C0
:1086E000109208081092070810920F0810920B08B9
:1086F00081E080937A050895EBEAF7E08AEF8787B7
:1087000086A38093E8078093FF0710927A05089567
:1087100081E080937A0508956F927F928F929F9265
:10872000AF92BF92CF92DF92EF92FF920F931F937F
:10873000CF93DF93CBEAD7E00CE817E0D8019E0196
:1087400040E050E0CA018555984F6C01FC018785D7
:10875000882391F06685082E000C990B860F911DD9
:108760008F3F910519F014F08FEF90E097FF02C052
:1087700080E090E0F6018687F901F080F3FE2AC0E0
:108780006581768111968D919C911297860F971F26
:1087900012969C938E931197F601E780EE2DF0E0F0
:1087A000EE0FFF1FE85FF147C590D490161617062D
:1087B00024F48C159D0530F40DC0672B59F0C816B4
:1087C000D90640F01296DC92CE9211978F2D877FBA
:1087D000F9018083495E5F4F295E3F4F16964C3505
:1087E000510509F0AFCF80917A05882309F4CCC0F8
:1087F00057E1F52E809107089091080820910D0807
:1088000030910E088217930709F0B9C02091100823
:1088100030911108B9016F5F7F4F70931108609319
:108820001008F90144914F3F79F5A9014E5F5F4F60
:108830005093110840931008FB0164916F3219F4B2
:1088400010927A059CC0663009F08CC0FA01449100
:10885000C90104969093110880931008F90133968A
:10886000E491E33529F490931308809312087AC0B9
:10887000E53409F077C08091120890911308909325
:108880001108809310086EC047FD40930B0890912B
:108890000B08892F8F7047FF08C02E5F3F4F309322
:1088A000110820931008FB014491907F903BE1F068
:1088B000903C09F451C0903909F054C0E09110087F
:1088C000F09111089F012F5F3F4F309311082093C3
:1088D00010082491220FF89EF0011124E555F84F5D
:1088E00060890E949B463EC0E0911008F0911108FB
:1088F0009F012F5F3F4F3093110820931008E491A0
:10890000473049F4F89ED0011124A555B84FEE0F19
:108910001C96EC9327C04B3049F4F89ED0011124EB
:10892000A555B84FEE0F1396EC931CC04C3549F487
:10893000F89ED0011124A555B84FEE0F1A96EC936E
:1089400011C0443679F4F89ED0011124A555B84FD2
:10895000EE0F1B96EC9306C0F89EF0011124E5552E
:10896000F84F408B80E198E00E94AB4590930E0851
:1089700080930D0810920808109207083BCF0196CB
:10898000909308088093070894EBA92E97E0B92EDE
:108990002EEBC22E27E0D22E3FEBE32E37E0F32E54
:1089A00066246A94712C888185FF42C02D893E8996
:1089B000232B09F43DC086FD3BC04701F2E08F1A2E
:1089C0009108D6019C91F401808198132EC0ED8905
:1089D000FE89BF016F5F7F4F7E8B6D8B84918F3FD0
:1089E00031F488818F7788831E8A1D8A1EC09F017B
:1089F0002E5F3F4F3E8B2D8BFB016491E82FF0E003
:108A0000EE0FFF1FE053FF4F25913491CE01F90186
:108A10000995ED89FE89CF0101969E8B8D8BE4919E
:108A2000D401EC93F6011082CCCF9F5FD6019C93CA
:108A3000988195FF6CC0F70180818F3F11F08F5FA7
:108A4000808397FD04C0F7013897908101C09FEFA4
:108A5000F70137978081882309F44EC03196508101
:108A6000552309F449C0992309F446C040910C08E4
:108A7000442309F441C0899FC00111249395892F93
:108A80009927589F9001599F300D1124C901939542
:108A9000892F99273B975081589F9001599F300DFE
:108AA00011243395232F3327429FC001439F900DFC
:108AB00011249395892F9927379620812223F1F04D
:108AC000D501EC91F0E0E050F047E491E0582E9FA2
:108AD000F0011124F395EF2FFF27A3014E1B5F0B2D
:108AE000489F9001499F300D589F300D1124C901B6
:108AF0009395892F992702C080E090E0F50130819D
:108B0000F70139972081230FD5012C9302C080E013
:108B100090E0F801808367960A5F1F4FF7E1AF0E80
:108B2000B11C87E1C80ED11C97E1E90EF11CA8E049
:108B3000C730DA0709F037CFDF91CF911F910F913E
:108B4000FF90EF90DF90CF90BF90AF909F908F906D
:108B50007F906F900895DC01ED91FC9111979F013A
:108B60002F5F3F4F11963C932E93E491E7FD03C096
:108B70008E2F90E00895EF778E2F90E09695982FA6
:108B80008827979587952F5F3F4FF9013197E4919B
:108B90004E2F4F77840F911DE7FDF0CF2D933C931F
:108BA0000895AF92BF92CF92DF92EF92FF920F9310
:108BB0001F93CF93DF931F92CDB7DEB75C01E62EF4
:108BC000FC018081F82FF078FF2EF50117869FEFCA
:108BD00096874587148A877B808312861186218336
:108BE000148293838281F9E06F9F80011124833086
:108BF00051F51092A1078091090890910A08800F01
:108C0000911FFC013196A591B491B093A307A09355
:108C1000A207AC01495F5F4FFA01C590D490059659
:108C2000FC0165917491C61AD70AD092A507C0922B
:108C3000A407FA0185919491A80FB91FB093A707D3
:108C4000A093A60705C060E029830E94EF46298112
:108C5000622FF50182810E94DB46F501FF2011F0B1
:108C6000E18A01C0E08AE0910908F0910A08E00F6A
:108C7000F11F339685919491F501009719F4168AA6
:108C8000158A08C0138AFC012491F501228B0196F4
:108C9000968B858B0F90DF91CF911F910F91FF9055
:108CA000EF90DF90CF90BF90AF900895CF93DF9378
:108CB000E0910908F0910A0899E0899FE00DF11D03
:108CC0001124E491E150E230D8F02091C20727FF4F
:108CD0001BC02091D307281302C0411115C0209159
:108CE000D90727FF0FC02091EA07281302C04111BE
:108CF00009C02091D6079091ED07921718F404C08F
:108D0000C3E003C0C2E001C0C1E097E1C99FE00138
:108D10001124C555D84F90E898831E8A1D8A20E5F6
:108D2000462F682FCE010E94D145888180628883BA
:108D3000DF91CF910895CF93DF93A82FB0E097E113
:108D4000899FF0011124E555F84F808185FF02C00D
:108D500087FD2EC0211118C097E19A9FF0019B9FBB
:108D6000F00D1124E555F84F9785911102C086FF4B
:108D7000158697E19A9FF0019B9FF00D1124E55510
:108D8000F84F8F7B808314C0822F242F97E19A9F06
:108D9000E0019B9FD00D1124C555D84F18821E8A23
:108DA0001D8A482FCE010E94D14588818062888328
:108DB000DF91CF91089599277727E8E0FEE8660FC5
:108DC000771FE60FF71FA591B491ECE8F7E026E0D6
:108DD000289FE00DF11DA183B283112408959927E6
:108DE0007727ECE8F7E026E0289FE00DF11D70E919
:108DF000760F75831124089581E080938B07089581
:108E000080E080938B07089522002400260028002C
:108E10002B002D0030003300360039003D004000AB
:108E2000440048004C00510056005B0060006600A2
:108E30006C00730079008100880090009900A20006
:108E4000AC00B600C100CC00D800E500F300010181
:108E5000100121013201440157016C018101980187
:108E6000B001CA01E5010202210241026402880246
:108E7000AE02D7020303300361039403CB0305045E
:108E800042048304C70410055D05AF0505066106AD
:108E9000C206290796070908830805098E09200AD2
:108EA000BA0A5D0B0A0CC10C840D510E2B0F121067
:108EB00007110A121D1340147415BA1614188319D9
:108EC000071BA31C571E24200E22142439267F289A
:108ED000E82A752D293006330F364539AD3C494017
:108EE0001B442848734CFE50CF55EA5A51600C661B
:108EF0001D6C8B725A79928037885090E598FDA14D
:108F00009FABD3B5A3C0000000000000000000002C
:108F10000000000000000000000000000000000051
:108F20000000000000000000000000000000000041
:108F30000000000000000000000000000000000031
:108F40000000000000000000000000000000000021
:108F50000000000000000000000000000000000011
:108F60000000000000000000000000000000000001
:108F700000000000000000000000000000000000F1
:108F800000000000000000000000000000000000E1
:108F900000000000000000000000000000000000D1
:108FA00000000000000000000000000000000000C1
:108FB00000000000000000000000000000000000B1
:108FC00000000000000000000000000000000000A1
:108FD0000000000000000000000000000000000091
:108FE0000000000000000000000000000000000081
:108FF0000000000000000000000000000000000071
:10900000000306090C101316191C1F2225282B2EED
:10901000313336393C3F414447494C4E5153555802
:109020005A5C5E60626466686A6B6D6F70717374BF
:10903000757678797A7A7B7C7D7D7E7E7E7F7F7F78
:109040007F7F7F7F7E7E7E7D7D7C7B7A7A7978765E
:1090500075747371706F6D6B6A68666462605E5C74
:109060005A585553514E4C494744413F3C39363389
:10907000312E2B2825221F1C191613100C0906034C
:1090800000FDFAF7F4F0EDEAE7E4E1DEDBD8D5D253
:10909000CFCDCAC7C4C1BFBCB9B7B4B2AFADABA81E
:1090A000A6A4A2A09E9C9A9896959391908F8D8C41
:1090B0008B8A888786868584838382828281818168
:1090C0008181818182828283838485868687888A62
:1090D0008B8C8D8F9091939596989A9C9EA0A2A42C
:1090E000A6A8ABADAFB2B4B7B9BCBFC1C4C7CACDF7
:1090F000CFD2D5D8DBDEE1E4E7EAEDF0F4F7FAFD14
:10910000808182838485868788898A8B8C8D8E8FE7
:10911000909192939495969798999A9B9C9D9E9FD7
:10912000A0A1A2A3A4A5A6A7A8A9AAABACADAEAFC7
:10913000B0B1B2B3B4B5B6B7B8B9BABBBCBDBEBFB7
:10914000C0C1C2C3C4C5C6C7C8C9CACBCCCDCECFA7
:10915000D0D1D2D3D4D5D6D7D8D9DADBDCDDDEDF97
:10916000E0E1E2E3E4E5E6E7E8E9EAEBECEDEEEF87
:10917000F0F1F2F3F4F5F6F7F8F9FAFBFCFDFEFF77
:10918000000102030405060708090A0B0C0D0E0F67
:10919000101112131415161718191A1B1C1D1E1F57
:1091A000202122232425262728292A2B2C2D2E2F47
:1091B000303132333435363738393A3B3C3D3E3F37
:1091C000404142434445464748494A4B4C4D4E4F27
:1091D000505152535455565758595A5B5C5D5E5F17
:1091E000606162636465666768696A6B6C6D6E6F07
:1091F000707172737475767778797A7B7C7D7E7FF7
:1092000000020406080A0C0E10121416181A1C1E6E
:1092100020222426282A2C2E30323436383A3C3E5E
:1092200040424446484A4C4E50525456585A5C5E4E
:1092300060626466686A6C6E70727476787A7C7E3E
:109240007F7D7B79777573716F6D6B69676563611E
:109250005F5D5B59575553514F4D4B49474543410E
:109260003F3D3B39373533312F2D2B2927252321FE
:109270001F1D1B19171513110F0D0B0907050301EE
:10928000FFFDFBF9F7F5F3F1EFEDEBE9E7E5E3E1DE
:10929000DFDDDBD9D7D5D3D1CFCDCBC9C7C5C3C1CE
:1092A000BFBDBBB9B7B5B3B1AFADABA9A7A5A3A1BE
:1092B0009F9D9B99979593918F8D8B8987858381AE
:1092C00080828486888A8C8E90929496989A9C9EAE
:1092D000A0A2A4A6A8AAACAEB0B2B4B6B8BABCBE9E
:1092E000C0C2C4C6C8CACCCED0D2D4D6D8DADCDE8E
:1092F000E0E2E4E6E8EAECEEF0F2F4F6F8FAFCFE7E
:109300007F7F7F7F7F7F7F7F7F7F7F7F7F7F7F7F6D
:109310007F7F7F7F7F7F7F7F7F7F7F7F7F7F7F7F5D
:109320007F7F7F7F7F7F7F7F7F7F7F7F7F7F7F7F4D
:109330007F7F7F7F7F7F7F7F7F7F7F7F7F7F7F7F3D
:109600000309131E28313A40464C5054585B5E61A2
:10961000636567696B6C6E6F707172737475767762
:10962000777879797A7A7B7B7C7C7C7D7D7D7E7E88
:109630007E7E7F7F7F7F7F7F7F7F7F7F7F7F7F7F3C
:109640007F7F7F7F7F7F7F7F7F7F7F7F7F7E7E7E2D
:109650007E7D7D7D7C7C7C7B7B7A7A79797877775F
:10966000767574737271706F6E6C6B696765636128
:109670005E5B5854504C46403A31281E1309030093
:10968000C6CCD5DBDFE3E5E7E9EAEBECEDEEEFEFA7
:10969000F0F0F0F1F1F1F1F2F2F2F2F2F2F2F2F3B3
:1096A000F3F3F3F3F3F3F3F3F3F3F3F3F3F3F3F38A
:1096B000F3F3F3F3F3F3F3F3F3F3F3F3F3F3F3F37A
:1096C000F3F3F3F3F3F3F3F3F3F3F3F3F3F3F3F36A
:1096D000F3F3F3F3F3F3F3F3F3F3F3F3F3F3F3F35A
:1096E000F2F2F2F2F2F2F2F2F1F1F1F1F0F0F0EF67
:1096F000EFEEEDECEBEAE9E7E5E3DFDBD5CCC60026
:1097000000283D42302D2C2B2C2D2E2F303233357E
:1097100037393B3D3F414345484A4C4E50535557DE
:10972000595B5D5F61636567696B6C6E70717374C3
:10973000757778797A7B7C7D7D7E7E7F7F7F7F7F6A
:109740007F7F7F7F7F7F7E7E7D7D7C7B7A79787750
:1097500075747371706E6C6B69676563615F5D5B77
:1097600059575553504E4C4A484543413F3D3B396C
:1097700037353332302F2E2D2C2B2C2D30423D28D7
:1097800000E9E5FED4D7D7D7D6D4D2D0CECCCAC83C
:10979000C6C3C1BFBDBAB8B6B4B1AFADABA9A7A57A
:1097A000A3A19F9E9C9A999795949391908F8D8C4D
:1097B0008B8A89888887868585848484838383834C
:1097C0008383838383848484858586878888898A44
:1097D0008B8C8D8F909193949597999A9C9E9FA135
:1097E000A3A5A7A9ABADAFB1B4B6B8BABDBFC1C34D
:1097F000C6C8CACCCED0D2D4D6D7D7D7D4FEE5E906
:10980000F9F8F9F5EBE1DDDEE0E2E4E5E6E5E4E2D6
:10981000DED9D2CAC1B7ACA299918A8683818080F1
:109820008182838586888A8C8D8F90929395969776
:1098300098999A9B9B9C9D9D9D9E9E9E9F9F9F9F5E
:109840009F9F9F9E9E9E9D9D9D9C9B9B9A99989756
:1098500096959392908F8D8C8A888685838281805D
:10986000808183868A9199A2ACB7C1CAD2D9DEE23F
:10987000E4E5E6E5E4E2E0DEDDE1EBF5F9F8F90048
:109880000708070B151F2322201E1C1B1A1B1C1E5A
:1098900022272E363F49545E676F767A7E7F7F7F20
:1098A0007F7E7D7B7A7876747371706E6D6B6A697A
:1098B0006867666565646463636262626161616171
:1098C000616161626262636363646565666768695A
:1098D0006A6B6D6E7071737476787A7B7D7E7F7F34
:1098E0007F7F7E7A766F675E54493F362E27221E31
:1098F0001C1B1A1B1C1E2022231F150B0708070008
:109900001F313D444E5354565A5F64696E747679E4
:109910007C7F7F7F7F7F7F7F7F7F7F7F7F7F7F7F5A
:109920007F7F7F7F7F7F7F7F7F7F7F7F7F7F7F7F47
:109930007F7F7F7F7F7F7F7F7F7F7F7F7F7F7F7F37
:109940007F7F7F7F7F7F7F7F7F7F7F7F7F7F7F7F27
:109950007F7F7F7F7F7F7F7F7F7F7F7F7F7F7F7F17
:109960007F7F7F7F7F7F7F7F7F7F7F7F7F7F7F7F07
:109970007F7F7F7F7F7F7F7F7F7F7F7C7871684C59
:109980002C1C120C0A0B0A05FDF3E9DFD4CAC0B780
:10999000AEA69E97918B8685828080808080808015
:1099A00080808080808080808080808080808080B7
:1099B00080808080808080808080808080808080A7
:1099C0008080808080808080808080808080808097
:1099D0008080808080808080808080808080808087
:1099E0008080808080808080808080808080808077
:1099F000808080808087919DACC4CBD4DDF2FAFA60
:109A000085E091E00E9431438EE091E00E94FF40AA
:109A10000E94D7408FE090E00E94A44D41E06FEF9C
:109A200080E00E9456464EE558E06CE082E10E94DC
:109A3000394D86E090E00E94A44D48E758E06CE084
:109A400082E10E94394D84E090E00E94A44D4EE5F1
:109A500058E06CE082E10E94394D80E490E00E9481
:109A6000A44D0E94D74084E190E00C94A44D089549
:109A700008954F925F926F927F928F929F92AF92D2
:109A8000BF92CF92DF92EF92FF920F931F93CF93EB
:109A9000DF93682E562E7A01FA01749031968490E5
:109AA000C72CD12C00E010E0912C9814F1F0C0E00C
:109AB000D0E05801F2E0AF0EB11C492C450CC7159F
:109AC00080F495012C0F3D1FF701E20FF31F249145
:109AD000422F50E0642D8C2F860D0E94E04021968D
:109AE000EECF93940C0D1D1DE0CFDF91CF911F9110
:109AF0000F91FF90EF90DF90CF90BF90AF909F902D
:109B00008F907F906F905F904F9008950F931F9369
:109B1000CF93DF93062FC42FD52F182F141BFE01D0
:109B20004491442349F04F774052602F8C2F810F8E
:109B30000E94ED402196F3CFDF91CF911F910F91BD
:109B4000089540520C94ED400F931F93CF93DF93F1
:109B50008C01C0E0D0E0C017D10744F40E9404415A
:109B60008823E1F30E9408412196F5CFDF91CF9140
:109B70001F910F910895CF92DF92EF92FF920F9372
:109B80001F93CF93DF9396E09093EA0820E130E0B3
:109B90003093CA082093C908E1ECF8E0108282E013
:109BA000F82EF182F28257E053834FEF448388E02E
:109BB00085831CE01683B7E1B783E1EAF8E020EF84
:109BC000208321EF21832FEE2283138271E074839F
:109BD00030E13583168277833087CFE0C18721E17A
:109BE000228713862EE0E22EE48622E125876FE1AC
:109BF000668761E26787108A518B428B4BE0438B0B
:109C0000948B858B63E0668B978B908F618F85E05B
:109C1000828F538FD4E0D48F858F668F978FE9E141
:109C2000F8E006E1008383E18183A5E1A283B383A9
:109C3000B4E1B483A58386830783BCE1CB2EC086C1
:109C4000A1873287BDE0B3871487B5873687A7879A
:109C5000208B218B228B238B248B258B268B278B90
:109C6000008FC18F8AE0D82ED28E538F948F558F5C
:109C7000768FC78F10A211A212A213A214A215A24E
:109C800016A217A220A741A792A763A7F4A665A7CB
:109C900096A747A710AA11AA12AA13AA14AA15AA2E
:109CA00016AA17AA30AF89E081AFD2AF73AF14AE56
:109CB00070935608D093570880935808109259080B
:109CC00010925A0810925B0810925C0810925D087E
:109CD00010925E0810925F0810926008309361083D
:109CE00080936208D09363087093640810926508AB
:109CF00070936608D093670880936808109269088B
:109D000010926A0810926B0810926C0810926D08FD
:109D100010926E0810926F081092700820937108CC
:109D2000409372089093730860937408F0927508DA
:109D30006093760890937708409378088093790829
:109D400080937A0880937B0880937C0880937D08B9
:109D500080937E0880937F08809380080093810819
:109D6000C0938208D092830850938408909385080A
:109D700050938608D0928708C0938808E09289089B
:109D800040938A08B0938B08C0938C0810938D0879
:109D9000B0938E0840938F08E0929008C09291088B
:109DA000A093920830939308B09394081093950869
:109DB000B093960830939708A0939808109299084A
:109DC000DF91CF911F910F91FF90EF90DF90CF9097
:109DD00008952091000130910101A901542F4427D9
:109DE000550F550F550FC9019695982F88279795B0
:109DF0008795840F951F820F931F96958795909353
:109E000001018093000108952F923F924F925F923B
:109E10006F927F928F929F92AF92BF92CF92DF927A
:109E2000EF92FF920F931F93CF93DF93CDB7DEB7DF
:109E3000CD54D1090FB6F894DEBF0FBECDBF3C01A3
:109E40007A8769874A012CA30E8BEBAA80E00E94D7
:109E50000E416C0181E00E940E418C299D29C09029
:109E6000D208D090D3088C299D299093D308809351
:109E7000D2088091E90891E0980F9093E908973013
:109E800024F08093E908C4019BC4830101501109A7
:109E90001A8F098F8091C9089091CA0818E181270B
:109EA0009093CA088093C9080E94E94E87778C87EF
:109EB00080E01E8221E030E049855A85241B350B65
:109EC00028963FAF2EAF28975195419551095CA731
:109ED0004BA77CA1672F70E0788F6F8B675E774F01
:109EE0002A967FAF6EAF2A97AF89B88DA058B10977
:109EF0002C96BFAFAEAF2C9755245394580EEBA9B8
:109F00008E1708F008C4BE81B078BD87E2E0E51581
:109F1000C0F4E52CF12CF3E0EF1AF10844275527A3
:109F20004819590900E010E020E830E028966EADAD
:109F30007FAD28978BA59CA50E94044F9A8B898B97
:109F400004C000E41FE11A8B098BA988BA88B19478
:109F5000A194B10829853A85A216B30634F0809100
:109F6000E7089091E80884974CF032E0351510F03E
:109F7000540104C0F0ECAF2EF0EEBF2E8091150816
:109F800090911608A0911708B09118080196A11D8C
:109F9000B11D8093150890931608A0931708B093ED
:109FA00018084C854F874A83652D70E024967FAF53
:109FB0006EAF249789899A8980549F4126969FAFD6
:109FC0008EAF26979A81C92ED12CF601E75EF74F06
:109FD000A081AF83EA2FF0E0FC8FEB8F8091C9085E
:109FE0009091CA088E239F23892B09F44FC3A77031
:109FF000A887AB830A2F10E01C8B0B8BF801EF5561
:10A00000F74F2089288B8A8130E1832790E0AC01CB
:10A01000475E574F5FAF4EAFB601625071097AA7E6
:10A0200069A76878772722967FAF6EAF229781E085
:10A030008D8B9885933008F41D8AAB81A7FF1BC3D5
:10A04000BD89BB2309F417C3A195AB838B8185958B
:10A0500087709A819D5F89278E8790E09EA78DA744
:10A0600081E0AE858A27E82FF0E0F8ABEFA782E029
:10A070008A27082F10E01AAB09AB2B893C892450A2
:10A0800031093EA32DA34B81042E000C550B58A77C
:10A090004FA34C0D5D1D5BAF4AAF5889852F90E0F3
:10A0A0000797282B392B3DAF2CAF4A8060E86B8790
:10A0B00070E87C838D85882309F445C04E8048264E
:10A0C00044C08AAD9BAD861997092F812072DC01AF
:10A0D000A22B9D01ECADFDADEF2B09F0C8C2EDA5A3
:10A0E000FEA5E75EF74F8081082E000C990B40918A
:10A0F000C9085091CA08841B950B069709F0B5C290
:10A10000E9A9FAA9E75EF74F9081EFA5F8A9E75E04
:10A11000F74F8081982B81E009F480E0FE85FB8772
:10A120001D898123A901482BCA01892B09F4A1C2E9
:10A1300081E05885553008F080E06D81680F69A393
:10A1400079A1711174CF9B81490E842D887809F013
:10A150006ECF2A96AEADBFAD2A978C91082E000C1B
:10A16000990B2C96EEADFFAD2C978E239F23892B58
:10A1700099F0842D90E02F89388D281B390B2230DF
:10A18000310554F40F89188D801B910B029724F42C
:10A19000E0E4AE2EEFE1BE2E61E01885133008F04A
:10A1A00060E02CA1421205C0662319F080E18425ED
:10A1B00001C0842D482F50E05E8F4D8FFA01E75E7D
:10A1C000F74F50815D8359A3E091C908F091CA0807
:10A1D000642C712C01E0511100E0802F90E0A3016C
:10A1E0004C195D094770552721E030E0452B11F0EF
:10A1F00020E030E0281B390B462F50E02423352384
:10A200007D81472F50E04E235F23242B352B2115D2
:10A21000310509F00CCF472F477050E04F53574F8F
:10A22000DA017C914D81407C50E01A01B5E27B025D
:10A23000200C311C112437FE04C070E4A72E7FE1EE
:10A24000B72E49855A85A416B50624F051E0551558
:10A2500008F423C271E0571206C0A101AB89BC8982
:10A260004A1B5B0B01C0A4012496AEADBFAD249781
:10A27000A81BB90B12970CF4E8C1B885B63098F456
:10A28000D601A75EB74F1896EC900E2C000CFF0875
:10A29000C301875E974FDC0118968C91E81AF1088C
:10A2A00087FDF39402C0E12CF12C5B85452F50E033
:10A2B0005BA34AA3C601875E974FDC011C928D8D7C
:10A2C0009E8D875E974FDC011C92CA01875E974F77
:10A2D000DC011C92C301875E974F4F814062DC0115
:10A2E0004C938B85887861F4BC818B2F90E0875EDE
:10A2F000974F46E04E0FDC014C93B2E3EB0EF11C9E
:10A300008091E7089091E80811E08E3191050CF4F6
:10A3100010E04DA15EA1412B452B11F424E130E06A
:10A32000E21AF30A662309F48AC0959587959595F4
:10A33000879522962EAD3FAD2297232BA1F429A518
:10A340003AA5275E374FD9012C91022E000C330B12
:10A3500051E040E06B8D7C8D2617370709F450E003
:10A36000252F342F02C021E030E0A6014E5F5F4F61
:10A37000BA0168787727672B91F4475E574FDA0167
:10A380004C91042E000C550B71E060E0AB8DBC8D40
:10A390004A175B0709F470E0472F562F02C041E0CF
:10A3A00050E0240F351F41E050E0421B530B9A014F
:10A3B000AEADBFAD4C91042E000C550BB49661E0D0
:10A3C00070E04E175F0711F060E070E0261B370B5E
:10A3D00069E0629FA001639F500D1124840F951FB7
:10A3E000E80EF91E8FA198A5860D971D019687FF8F
:10A3F00007C027E832E0EB89FC892E1B3F0B09C020
:10A400002F81207230E0C301409628233923220F88
:10A41000331FF301E75EF74F8081820F8083220EA6
:10A42000331E9091DD089E3431F0923531F0923434
:10A4300031F4825003C0845001C081508083C40134
:10A44000820D931D9701280F391F2E963FAF2EAF17
:10A450002E97B8A2AF8E498D5A8DA416B50614F466
:10A4600058A34F8F81E052E0551508F480E0B12FDA
:10A47000B82B26968EAD9FAD26978B2B892B99F006
:10A480002FEF250D81E065E0651508F080E09D89DE
:10A49000982381E07D85711180E08923A02FA82376
:10A4A0002A1B298301C059829C81892F90E09DAB92
:10A4B0008CAB2E96AEADBFAD2E97B195A195B109DF
:10A4C000BFABAEABEF8DF8A1F195E195F109F9AF16
:10A4D000E8AFF981F33048F42E960EAD1FAD2E97FC
:10A4E0002F8D38A1201731079CF43981E32EF12CF0
:10A4F00000E010E02CA93DA94EA95FA968AD79AD97
:10A500008BA59CA50E94044F91958195910904C04B
:10A510002E968EAD9FAD2E9749814F5F4983698DF1
:10A520007A8D6817790714F4451598F2AC017E8985
:10A53000772309F46DC060919D0870919E08603486
:10A54000AFE17A07A9F1803CB0EE9B0789F1C6160E
:10A55000D70671F52091E408022E000C330B621629
:10A56000730631F588279927881999098219930963
:10A570009093A00880939F08EC818E2F90E0909399
:10A58000E3088093E208C101880F892F881F990B87
:10A590002091E7083091E808820F931F9093E80814
:10A5A0008093E7088091E90881508093E9082CC0E6
:10A5B000FE89F93069F52091CB08211129C040911D
:10A5C000E408042E000C550B31E06416750609F002
:10A5D00030E021E0C616D70609F020E02323B9F0C9
:10A5E000803C904EA1F088279927881999098219F3
:10A5F00093099093A00880939F081C81812F90E07D
:10A600009093E3088093E20889859A85D9C0A501D3
:10A61000EAA1FBA1E75EF74F8091C9088A5F8083BA
:10A62000F301E75EF74F10822C81E22FF0E0E75E46
:10A63000F74F1082F601E75EF74F3F813083ED8DD3
:10A64000FE8DE75EF74F6D816083A416B5063CF47E
:10A650008C81807884298E837A817F875A018D85C9
:10A66000882309F42ECD1D8620CD0E850B8781E031
:10A6700057CD4C8265CDE889EF5FE88BF0E0EF5570
:10A68000F74F808181958B838111E0CC8A81875F30
:10A6900087778A83FC858F1395CCC5018854914EAA
:10A6A00081379D4310F092E6592E9501205C304E83
:10A6B00081E090E049895A8940345F4111F080E09F
:10A6C00090E0822B932B892B11F4A12CB12C7E8945
:10A6D0007723E9F082E08515D0F48F8587708F5954
:10A6E0008093D9089F8592959F7088E3A82FA91B16
:10A6F000A093DA089E8197709F599093DB089E8102
:10A7000092959770891B8093DC081092DD08852D47
:10A71000BF85BC87F1CBF2E0F51508F0F4CB0E89CC
:10A72000202F30E081E090E040919D0850919E08FC
:10A7300040345F4111F080E090E082239323892B25
:10A7400039F121E62515B0F0409115085091160811
:10A7500060911708709118088091CE089091CF08E9
:10A76000A091D008B091D108481759076A077B0714
:10A770000CF4C9CB3C85832F90E090939E08809386
:10A780009D088E8187778093E40883E0582EBBCBA9
:10A790008091C9089091CA0848E184279093CA081B
:10A7A0008093C9088091E90881508093E90881E08D
:10A7B00090E0A814B90414F080E090E08A0D9B1D8D
:10A7C000C35BDF4F0FB6F894DEBF0FBECDBFDF9186
:10A7D000CF911F910F91FF90EF90DF90CF90BF909E
:10A7E000AF909F908F907F906F905F904F903F9031
:10A7F0002F900895CF92DF92EF92FF920F931F93C5
:10A80000CF93DF931092D3081092D208C0E4DFE117
:10A8100080EFD82ECC24C3940E94E85B0E94BE59DE
:10A82000882329F08091D808811160C05BC00E9404
:10A8300032590E940357D0939E08C0939D082091DF
:10A84000D9082A30D1F08091DA0830EF8302C001B4
:10A850001124820F911D27FD9A95815E9C4F909344
:10A860009E0880939D088091DB08815E9091DC08B2
:10A870009D9D800D11248093E4081092150810927C
:10A88000160810921708109218080E94C15B809158
:10A89000D2089091D30882FD05C0892B29F08091C0
:10A8A000CC088111C092D8088091D8088111BACF04
:10A8B000E090EA080E2C000CFF082091E20830918D
:10A8C000E30840919F085091A00809E010E060E47F
:10A8D0007FE180EC90EE0E94044F823C904E0CF0A1
:10A8E0009BCFA0CF8091CC088823A1F080E00E946C
:10A8F0000E41892BD9F781E00E940E41892BB1F7D7
:10A90000DF91CF911F910F91FF90EF90DF90CF904B
:10A910000C94E85B0E94E85B81E08093CB0888E7B9
:10A920008093D9088093DB08DF91CF911F910F911D
:10A93000FF90EF90DF90CF900C94325990919C084B
:10A9400090FF04C041E06FEF0C94564608952091AB
:10A950009C0821FD0C94534308952F923F924F92EF
:10A960005F926F927F928F929F92AF92BF92CF929F
:10A97000DF92EF92FF920F931F93CF93DF9388E9BB
:10A9800098E00E94FF408CE60E94FC400E94D74065
:10A990000E94FC461092CC08C0E0D0E048E5E42ECE
:10A9A00042E0F42E512C51E1452E81E090E00E94CE
:10A9B000A44D48E05FE260E080E00E94394D4FEB3B
:10A9C0005BE764E170E08CE090E00E94864D46EC2D
:10A9D0005BE765E170E08CE090E00E94864D4DEC15
:10A9E0005BE766E170E08CE090E00E94864D44ED0C
:10A9F0005BE767E170E08CE090E00E94864D4BEDF4
:10AA00005BE768E170E08CE090E00E94864D42EEEA
:10AA10005BE76AE170E08CE090E00E94864D409137
:10AA2000CD08449EA00111244F5A544864E170E0BF
:10AA300083E190E00E94864D4091E008449EA00191
:10AA400011244F5A544865E170E083E190E00E9480
:10AA5000864D80919C0880FB222420F8312CA10196
:10AA6000440F551F440F551F4954544866E170E088
:10AA700083E190E00E94864D80919C0881FB6624D2
:10AA800060F8712CA301440F551F440F551F495402
:10AA9000544867E170E083E190E00E94864D809128
:10AAA0009C0882FBCC24C0F8D12CA601440F551F72
:10AAB000440F551F4954544868E170E083E190E029
:10AAC0000E94864D652D70E06C5E7F4F46EF5BE720
:10AAD0008AE090E00E94864DCD2B79F080E00E94C4
:10AAE0000E41EC0181E00E940E418C2B9D2B892BA5
:10AAF000A9F788E5E82E82E0F82E80E00E940E415A
:10AB0000EC0181E00E940E41C82BD92BC4FF08C084
:10AB1000552019F05A948FE101C080E20E949E54A2
:10AB20004E01E0E48E2299245E01F0E8AF22BB24BE
:10AB3000C5FF0FC0E3E0E51540F053948FE10E949C
:10AB40009E54F1E05F1228C009C080E20E949E542A
:10AB500023C081E0851500F1552029F05524539438
:10AB600000EE18E002C00DEC18E0892859F0F80159
:10AB70008081882321F0815080838FE101C080E2B1
:10AB80000E949E54AB28E1F1F80180818530A8F540
:10AB90008F5F80838FE132C001E010E08EEF850D82
:10ABA00001C0000F8A95EAF78928A1F080919C08DE
:10ABB000982F902361F0802780939C088FE10E945A
:10ABC0009E54F3E05F1206C00E947C4303C080E203
:10ABD0000E949E54AB28A1F080919C08982F90234E
:10ABE00061F4082700939C088FE10E949E5483E043
:10ABF000581206C00E94884303C080E20E949E54FF
:10AC0000E1E0EE1AF108C3FD05C0E114F10409F01A
:10AC1000CCCE02C0EF28B1F481E08093CC08DF9164
:10AC2000CF911F910F91FF90EF90DF90CF90BF9049
:10AC3000AF909F908F907F906F905F904F903F90DC
:10AC40002F90089580E00E940E41EC0181E00E9467
:10AC50000E418C2B9D2B83FDF5CF80919C0883703A
:10AC600019F00E94FC4602C00E94004781E2DF9179
:10AC7000CF911F910F91FF90EF90DF90CF90BF90F9
:10AC8000AF909F908F907F906F905F904F903F908C
:10AC90002F900C949E548CE49AE30E94FF4080E233
:10ACA0000E94FC400E94D7404CEF5FE560E080E0EE
:10ACB0000E94394D8FEF8093E5088093E1088091E1
:10ACC000E008823018F480E68093E5088091CD0892
:10ACD000823018F480E18093E1088FEF8093D608EA
:10ACE0008093E60880E28093EC0880E18093D708A7
:10ACF0001092CB081092D5081092D40884E6809365
:10AD0000ED081092D8080C94BB4DFF920F931F933F
:10AD1000CF93DF93EC01F62E80E00E940E418C0170
:10AD200081E00E940E41802B912B82FF05C081E0C3
:10AD30008093D80880E061C08F2D0E940E418C0165
:10AD4000807F9927892BB1F106FF0BC09881892F4D
:10AD5000877021F0915098838FE101C080E20E94BA
:10AD60009E5407FF0CC09881892F8770873021F08F
:10AD70009F5F98838FE101C080E20E949E5404FF90
:10AD80000BC09881892F807721F0905198838FE1B3
:10AD900001C080E20E949E5405FF0CC09881892F5B
:10ADA0008077803721F0905F98838FE101C080E247
:10ADB0000E949E5488818093D60803701F70012BD7
:10ADC00079F081E20E949E548F2D0E940E41837083
:10ADD0009F70892B19F00E943259F6CF88810DC0DF
:10ADE0001BE08F2D0E940E41892B21F00E943259C9
:10ADF0001150B9F70E9432598FCFDF91CF911F9137
:10AE00000F91FF900895CF92DF92EF92FF920F93F0
:10AE10001F93CF93DF938FEF8093D6088093E6083C
:10AE20008091C90884FF07C0C091E00895EEC92E43
:10AE300098E0D92E06C0C091CD0881EEC82E88E0DA
:10AE4000D82EC23030F48091CC08811104C00FEFAD
:10AE500098C0C23021F08091CC08882301F180E2B3
:10AE600090E0A0E0B0E08093CE089093CF08A0934C
:10AE7000D008B093D10883E08093EA081092C1080B
:10AE800081E08093C2088093C3088093C4089FEF39
:10AE90009093C5088093C6088093C70845C0C33007
:10AEA00071F480E490E0A0E0B0E08093CE0890934D
:10AEB000CF08A093D008B093D10884E01FC0C4305D
:10AEC00071F480E890E0A0E0B0E08093CE08909329
:10AED000CF08A093D008B093D10885E00FC0C5304B
:10AEE00029F580E094E0A0E0B0E08093CE08909354
:10AEF000CF08A093D008B093D10886E08093EA08E9
:10AF00001092C10882E08093C2088093C30887E052
:10AF10008093C4088FEF8093C50888E08093C608AB
:10AF20008CE08093C70887E18093C8080E9432595B
:10AF300081E08093CB088AE08093D9081092DA08E8
:10AF40008BED98E090939B0880939A0843C1809181
:10AF5000D808811103C080E20E949E54F70120812D
:10AF60002871022E000C330B8091C9089091CA08F9
:10AF7000F8E18F274091D80828173907E1F04111EF
:10AF80001AC06C2FC6010E948556D82F90E09C01F4
:10AF9000275E374F7901F90180818871082E000CF6
:10AFA000990B2091C9083091CA08F8E12F27821720
:10AFB000930769F6D3CF41110DC1D093E6080E94E3
:10AFC00032596C2FC6010E948556182F0093D6085F
:10AFD0000093E6080E9432598091D8081D1302C0E0
:10AFE000882379F28111F6C083E08093EA083D2F2F
:10AFF00037703F593093D908D077D295DF7098E3F6
:10B00000492F4D1B4093DA08212F27702F59209389
:10B01000DB08107712951F70892F811B8093DC0845
:10B020009AE09093DD081092DE086FED78E070935F
:10B030009B0860939A083093EE084093EF082093A2
:10B04000F0088093F108F70120812770022E000C90
:10B05000330B215031092230310508F0BBC0813358
:10B0600019F0883309F0B6C0D0E01AE940EB54E695
:10B070006CE088E00E94394D81E090E02091DC088E
:10B08000213311F080E090E0189FA001199F500D2E
:10B090001124475B55486DE089E00E94394D81E0FD
:10B0A00090E02091DC08213311F080E090E0189FBF
:10B0B000A001199F500D11244D5C55486DE08CE0A6
:10B0C0000E94394D81E090E02091DC08213311F09D
:10B0D00080E090E0189FA001199F500D1124485D59
:10B0E00055486DE08FE00E94394D81E090E020915D
:10B0F000DC08213311F080E090E0189FA001199F37
:10B10000500D1124425C55486DE082E10E94394D9A
:10B110008091EB0883FF09C08D2F880F8D0F46E4C7
:10B120005BE76DE0875F0E94394D81E090E00E940F
:10B13000A44D8091EB088F5F8093EB088C2F0E94C9
:10B140000E4186FF0FC0DD2351F0D1508FE10E94E8
:10B150009E548C2F0E940E4186FDFBCF03C080E2DF
:10B160000E949E548C2F0E940E4187FF0FC0D33047
:10B1700050F4DF5F8FE10E949E548C2F0E940E419D
:10B1800087FDFBCF03C080E20E949E548C2F0E945B
:10B190000E4183709F70892B09F468CF81E20E9471
:10B1A0009E548C2F0E940E41892BD9F7D23031F05A
:10B1B000D33031F0D13031F48EE405C082E503C0E4
:10B1C00082E401C081E58093DD088AE08093DE0897
:10B1D0001092DF08DF91CF911F910F91FF90EF90B8
:10B1E000DF90CF900895342F90E0E62FF0E0DC015F
:10B1F000AE1BBF0BA170BB277DE47A9FA0017B9F94
:10B20000500D11247BE0379F400D511D11243AE968
:10B21000239F400D511D11244E5E55489F0174E03F
:10B22000220F331F7A95E1F7280F391FE091D608D6
:10B23000F0E0E217F30731F0E091E608F0E0E21702
:10B24000F30731F42091EB0823FF02C046E45BE7EB
:10B25000262F220F620F6E5F0196982F990F890F8C
:10B260000C94394DDF92EF92FF920F931F93CF937F
:10B27000DF938091EB088F5F8093EB0881E090E093
:10B280000E94A44D89E1E82E88E0F82ED12CD0E070
:10B29000C0E000E010E0802FF701E00FF11F908187
:10B2A000E92FE7704E2FEE0F550B660B770BFA0167
:10B2B0003197E730F105B0F4E85CFF4FCF5F0C94B5
:10B2C000BC5C41E010C0DF5F43E00DC0DF5F46E0E3
:10B2D0000AC0DF5F44E007C0DF5F42E004C0DF5F19
:10B2E00045E001C040E021E093FD20E06D2D0E948B
:10B2F000F3580F5F1F4F0830110569F6D39480E1B2
:10B30000E80EF11C88E0D812C4CF8091CC088823C5
:10B31000C1F04BEB50E06AE180E20E94E0404CEB70
:10B3200050E06AE181E20E94E04046EC50E06AE1D0
:10B3300082E20E94E04047EC50E06AE183E20E9432
:10B34000E0408091EC08C81730F484E20E949E54DB
:10B3500084E68093ED088091D7088D1718F485E274
:10B360000E949E54C093EC08D093D708DF91CF91F0
:10B370001F910F91FF90EF90DF900895CF92DF9291
:10B38000EF92FF920F931F93CF93DF938091D40896
:10B390009091D508009739F481E090E09093D5081A
:10B3A0008093D408E3C1D091CB08D1111CC0309157
:10B3B000EE082091D908321312C03091EF08209185
:10B3C000DA0832130CC03091F0082091DB083213F8
:10B3D00006C03091F1082091DC08321721F082E29A
:10B3E0000E949E54C4C1EC012196D093D508C0930D
:10B3F000D408CA31D105F0F081E090E00E94A44D5C
:10B400008EE191E06CE0680F20E030E0AC01420F8B
:10B41000531FFA01E858FF4F7081B8977083285D79
:10B420003F4F203C43E0340789F701966813ECCF87
:10B43000C9E1D0E08091DB089091DC08E8E3F0E01E
:10B44000E91BF10997FDF39564E0EE0FFF1F6A9584
:10B45000E1F7E80FF11D87FDFA95E854F84F808178
:10B460008770082E000C990B0197029718F484E658
:10B470008093ED088091ED0881508093ED088091D4
:10B48000D4089091D50880FD36C09695879568EED2
:10B4900073E00E94945CFC2E5AE0C52ED12CB601BC
:10B4A0000E94A85C8B01AC0142555F4F6C2F8EE16E
:10B4B0000E94E0400115110559F0C801B6010E9433
:10B4C000A85CAC0142555F4F6C2F8DE10E94E040BB
:10B4D0002AE030E0C801B9010E94A85CCB010097C6
:10B4E00051F0B9010E94A85CAC0142555F4F6F2D2D
:10B4F0008CE10E94E0404091D908495ABE0180E2A7
:10B5000090E00E94A14D4091DA084258BE0181E2CC
:10B5100090E00E94A14D4091DB08495ABE0182E2B1
:10B5200090E00E94A14D4091DC084258BE0183E2A8
:10B5300090E00E94A14D8091CB08882309F448C077
:10B540008091D908815698E32091DA08392F321B6F
:10B5500040E1349F800D11248093D6088091DB0850
:10B5600081562091DC08921B20E1929F800D1124CE
:10B570008093E60883E20E949E543CE3F32E0E94EF
:10B58000325980E00E940E418C0181E00E940E4100
:10B59000802B912B0091D2081091D308802B912BF6
:10B5A0009093D3088093D208FA94F110E8CF8FEFEC
:10B5B0008093D6088093E6080E9432598091CB0888
:10B5C000882321F08091ED0887FDB5C01092CB084B
:10B5D0008091DD08813531F440EC50E06C2F84E23D
:10B5E0000E94E0408091DD08823531F442EC50E069
:10B5F0006C2F84E20E94E0408091DD08823431F4B7
:10B6000043EC50E06C2F84E20E94E0408091DD0822
:10B610008E3431F441EC50E06C2F84E20E94E04023
:10B6200084E08093EA088091C9089091CA0838E1C3
:10B6300083279093CA088093C908EE24E394F12CE1
:10B6400000E810E020E830E040E050E060E47FE116
:10B6500080EC90EE0E94044F8C0180349F41E1F514
:10B6600044EC50E06C2F85E20E94E04086E20E94AC
:10B670009E542091C9083091CA0888E12827309348
:10B68000CA082093C90810939E0800939D0893E070
:10B69000E92EF12C00E810E020E830E040E050E036
:10B6A00060E47FE180EC90EE0E94044F823C904E7B
:10B6B00044F444EC50E06C2F86E20E94E04087E2C4
:10B6C00047C08091C9089091CA0838E183279093B8
:10B6D000CA088093C90840C08091C9089091CA08DF
:10B6E00048E184279093CA088093C90883E0E82E34
:10B6F000F12C00E810E020E830E040E050E060E4A9
:10B700007FE180EC90EE0E94044F8091C9089091F7
:10B71000CA0828E182279093CA088093C9089091AB
:10B72000D9088091DB08981317C09091DA088091AE
:10B73000DC08981311C045EC50E06C2F85E20E94A4
:10B74000E04045EC50E06C2F86E20E94E04088E249
:10B750000E949E54D1E00BC08091C9089091CA0804
:10B7600038E183279093CA088093C908D0E08D2FD1
:10B77000DF91CF911F910F91FF90EF90DF90CF90CD
:10B78000089580919C0882FF22C08091CB08882375
:10B79000F1F08091CC0881111AC081E090E00E9404
:10B7A000A44D61E081E00E94394181E090E00E9477
:10B7B000A44D8AE693E30E94FF404AEF59E360E01C
:10B7C00080E00E94394D60E18EE60C943941089585
:10B7D00080919C0882FF1AC081E090E00E94A44DF5
:10B7E00061E081E00E94394181E090E00E94A44D37
:10B7F0008CE49AE30E94FF404EE554E660E080E06E
:10B800000E94394D60EE84E10C9439410895CF9344
:10B81000DF93CDB7DEB7A0970FB6F894DEBF0FBEAB
:10B82000CDBF8FE996E60E9431431092E00882E096
:10B830008093CD0883E080939C08109201011092C0
:10B840000001BE016F5F7F4F80E890E00E940742D9
:10B85000811117C08B81982F92959F709093E0086B
:10B860008F708093CD088C818F7080939C088D8120
:10B8700090E0982F88272E81822B9093010180934E
:10B88000000180E8E82EF12C0E94AD54FA82E98292
:10B890008091E00820E1829FC00111249091CD08A1
:10B8A000892B8B8380919C088C831D828091000161
:10B8B0008E83CE0101960E94BD418091CC088111FA
:10B8C00004C080E198E60E94A7540E944B560E9453
:10B8D000FA538091D808882349F08091CC088823B6
:10B8E00001F180EF90E00E94A44D1BC08091CC0834
:10B8F0008111F3CF80E00E940E418C0181E00E9413
:10B900000E41802B912B892BA9F780E00E940E41DC
:10B910008C0181E00E940E41802B912B892BA9F391
:10B92000DCCF0E947C43B0CFAA1BBB1B51E107C0F8
:10B93000AA1FBB1FA617B70710F0A61BB70B881FBF
:10B94000991F5A95A9F780959095BC01CD0108954E
:10B9500097FB072E16F4009407D077FD09D00E94BC
:10B96000945C07FC05D03EF4909581959F4F089517
:10B97000709561957F4F0895EE0FFF1F0590F4912C
:08B98000E02D0994F894FFCFBB
:02B988000100BC
:00000001FF
